:100000000C94F7060C941F070C941F070C941F0701
:100010000C941F070C941F070C941F070C941F07C8
:100020000C941F070C9423090C9463320C94DE3259
:100030000C941F070C941F070C941F070C941F07A8
:100040000C94E60D0C941F070C941F070C941F07CB
:100050000C941F070C941F070C941F070C948629FF
:100060000C941F070C94802E0C94BB2E0C941F072D
:100070000C941F070C941F070C941F070C941F0768
:100080000C941F070C941F070C941F070C941F0758
:100090000C941F070C941F070C941F070C941F0748
:1000A0000C941F070C941F070C941F073C1D431D45
:1000B000431D3C1D431D431D431D431D431D431D47
:1000C000431D431D431D431D431D431D431DAB1CC9
:1000D000431D431D431D431D431D0E1C431D431D56
:1000E000431D431D431D431D431D431D431D431D10
:1000F000431D431D431D431D431DB71CB71CB71CA7
:10010000B71CB71CB71CB71CB71CB71C431D431D3D
:10011000431D431D431D431D131CB61CB61CB61CBA
:10012000B61C431DCD1CD51CDD1CE51CED1CF51CAF
:10013000FD1C051D0F1D191D231D2D1D5A1C1A1CEC
:10014000431D431D431D431DAB1C431D431D431D48
:10015000431D431D431D431D431DB51CB51CB51C4C
:10016000B51C431DCD1CD51CDD1CE51CED1CF51C70
:10017000FD1C051D0F1D191D231D2D1D5A1C1A1CAC
:10018000431D431D431D431DAB1C456E746572200A
:100190006D656E752E2E2E00546F67676C6564203A
:1001A0006D6963726F50504D00546F67676C656482
:1001B00020696E7665727465642050504D2100543C
:1001C0006F67676C6564205458206D7574696E673D
:1001D0002100546F67676C65642074656C656D659C
:1001E000747279210050726F746F636F6C20657246
:1001F000726F7220776974682052580054696D6577
:100200006F7574207768656E20636F6E6E656374BA
:10021000696E6720746F20525800507265737320A6
:10022000616E79206B657920746F2063616E636500
:100230006C00436F6E6E656374696E6720746F2027
:1002400052582C20706F7765722075702074686525
:100250002052582028776974682062696E64207083
:100260006C7567206966206E6F74207573696E67A0
:1002700020616C776179732062696E642900546F24
:1002800067676C65642027696D6D65646961746575
:10029000206F75747075742700546F67676C6564A0
:1002A0002027736C617665206D6F64652700546F3D
:1002B00067676C65642027616C7761797320626978
:1002C0006E642700546F67676C65642050504D2042
:1002D0006368616E6E656C206C696D69740053654E
:1002E00074205253534920696E6A656374696F6E56
:1002F000206368616E6E656C2028303D3D646973D3
:1003000061626C6529005365742050504D206D6901
:100310006E696D756D2073796E630053657420622C
:100320006561636F6E20696E74657276616C0053EF
:10033000657420626561636F6E2064656C6179002D
:1003400053657420626561636F6E206672657175B6
:10035000656E637920696E20487A3A20303D646981
:100360007361626C652C2050783D504D522063685B
:10037000616E6E656C20782C2046783D4652532085
:100380006368616E6E656C20780053657420505709
:100390004D2073746F702064656C61792028302063
:1003A00064697361626C65642C20312D32353520AF
:1003B0003D3D20302E3173202D2035306D696E2962
:1003C000005365742050504D2073746F7020646525
:1003D0006C61792028302064697361626C65642CDB
:1003E00020312D323535203D3D20302E3173202DEA
:1003F0002035306D696E2900536574206661696C23
:10040000736166652064656C6179202830206469B9
:100410007361626C65642C20312D323535203D3D91
:1004200020302E3173202D2035306D696E29002A41
:100430002A2A2A2A2A2A2A2A2A2A2A2A2A2A2A2A1C
:100440002A2A2A2A2A2A2A2A2A2A2A2A00525820EA
:1004500041636B6564202D2072657665727420732C
:1004600075636365737366756C21002A2A2A2A2ACC
:100470002A2A2A2A2A2A2A2A2A2A2A2A2A2A2A2ADC
:100480002A2A2A2A2A2A2A2A002A2A2A2A2A2A2AF6
:100490002A2A2A2A2A2A2A2A2A2A2A2A2A2A2A2ABC
:1004A0002A2A2A2A2A2A0052582041636B6564208E
:1004B0002D20757064617465207375636365737353
:1004C00066756C21002A2A2A2A2A2A2A2A2A2A2AF6
:1004D0002A2A2A2A2A2A2A2A2A2A2A2A2A2A2A2A7C
:1004E0002A2A0056616C69642063686F69636573CA
:1004F000206172653A205B315D2D5B31365D2028CD
:100500006368616E6E656C20312D3136290053654C
:1005100074206F757470757420666F7220706F72BE
:100520007420005B585D2061626F727420636861A3
:100530006E67657320616E64206578697420525817
:1005400020636F6E666967005B535D20736176653B
:100550002073657474696E677320746F205258003D
:100560005B525D2072657665727420525820736507
:100570007474696E677320746F2064656661756C4E
:10058000747300557365206E756D62657273205BC0
:10059000312D445D20746F206564697420706F7222
:1005A0007473205B452D515D20666F7220736574F6
:1005B00074696E677300202D2072656365697665C6
:1005C0007220636F6E666967757261746F722C203A
:1005D000727820737720000A0A6F70656E4C525350
:1005E0006E6720005365742073657269616C2062C8
:1005F000617564726174653A200056616C696420AB
:1006000063686F696365733A2031202D20342B3481
:10061000202F2032202D2038202F2033202D20384D
:100620002B34202F2034202D203132202F20352034
:100630002D2031322B34202F2036202D2031360032
:10064000536574204368616E6E656C20636F6E66DF
:1006500069673A2000536574204461746172617463
:10066000652028302D32293A200053657420486FC8
:1006700070206368616E6E656C7320286D617820F0
:1006800032342C2073657061726174656420627904
:1006900020636F6D6D6173292076616C69642076CB
:1006A000616C75657320312D3235353A2000536504
:1006B00074206368616E6E656C2073706163696E2F
:1006C0006720287831306B487A293A2000536574C6
:1006D00020524620706F7765722028302D37293AD6
:1006E0002000536574205246206D6167696320289D
:1006F0006865782920652E672E203078444541446E
:10070000463030443A20005365742062617365209E
:100710006672657175656E63792028696E20487A06
:10072000293A20005B5A5D20656E746572207265FF
:1007300063656976657220636F6E6669677572615D
:1007400074696F6E207574696C79005B465D206416
:100750006973706C61792061637475616C20667275
:10076000657175656E636965732075736564005B9B
:10077000525D2063616C63756C6174652072616E9B
:10078000646F6D206B657920616E6420686F7020E6
:100790006C697374005B495D207265696E69746988
:1007A000616C697A652073657474696E677320740F
:1007B0006F20736B657463682064656661756C7423
:1007C00073005B585D2072657665727420636861A2
:1007D0006E67657320616E642065786974206D654D
:1007E0006E75005B535D207361766520736574746C
:1007F000696E677320746F20454550524F4D2061DC
:100800006E642065786974206D656E75005573653A
:10081000206E756D62657273205B302D395D2074BA
:100820006F206564697420706172616D65746572B2
:100830007300202D2053797374656D20636F6E668D
:10084000696775726174696F6E000A0A6F70656E10
:100850004C52536E6720005129204F757470757487
:10086000206265666F7265206C696E6B20283D465C
:100870005329203A2000502920536C617665206D61
:100880006F646520286578706572696D656E746146
:100890006C293A20004F292054696D656420424933
:1008A0004E44206174207374617274757020203A14
:1008B00020004E292050504D206F757470757420A3
:1008C0006C696D6974656420202020203A20004402
:1008D000495341424C4544004D292050504D20522F
:1008E00053534920746F206368616E6E656C2020DD
:1008F00020203A20004C292050504D206D696E690F
:100900006D756D2073796E63202875732920203AE8
:10091000200044495341424C4544004B2920466144
:10092000696C7361666520626561636F6E20696ED4
:1009300074762E2028312D32353573293A20004A1D
:1009400029204661696C7361666520626561636F29
:100950006E2064656C61792028302D323535203D5C
:100960003E20313073202D203135306D696E293AAB
:1009700020004929204661696C73616665206265C3
:1009800061636F6E206672712E203A200048292024
:1009900050574D2073746F702064656C617920200E
:1009A00020202020203A200047292050504D20733D
:1009B000746F702064656C617920202020202020D5
:1009C0003A20004629204661696C7361666520649F
:1009D000656C6179202020202020203A200050578B
:1009E0004D206368616E6E656C200066756E637481
:1009F000696F6E3A20002920706F72742000445491
:100A000046205548462033322D62697420313063C8
:100A100068004F70656E4C52536E675258206D6976
:100A20006E6920342F36636800466C7974726F6E7D
:100A30002F4F72616E6765525820554846203863C3
:100A40006800525820747970653A200044697361D7
:100A5000626C656400487A00203D3D200043616C73
:100A600063756C61746564207061636B6574206983
:100A70006E74657276616C3A20004229204D69637C
:100A8000726F202868616C66292050504D2020200C
:100A9000203A00412920496E7665727465642050C1
:100AA000504D20696E20202020203A003029204D12
:100AB0007574652062757A7A657220286D6F73741B
:100AC0006C79293A0039292053657269616C20627A
:100AD000617564726174653A00736D617274506F10
:100AE0007274004672536B79005472616E73706158
:100AF00072656E740044697361626C6564003829C4
:100B00002054656C656D657472793A202020202030
:100B10002020003729204368616E6E656C20636F6A
:100B20006E6669673A20200036292044617461723C
:100B30006174652028302D32293A20202000352983
:100B400020486F70206368616E6E656C733A202078
:100B5000202020003429204368616E6E656C20736C
:100B6000706163696E673A20200033292052462065
:100B7000706F7765722028302D37293A20202000A9
:100B80003229205246206D616769633A2020202077
:100B900020202020200031292042617365206672C8
:100BA000657175656E63793A2020200000000000B1
:100BB000240027002A002D0030000000000025003E
:100BC00028002B002E00310000000000230026002A
:100BD00029002C002F00040404040403040502026D
:100BE00002020403020202020606060606060404C6
:100BF00002020204040802011040804010204080DC
:100C00004080080204018040201002011080102062
:100C100040400000000200080E0000030401000B29
:100C200000000000000000000000000000000000C4
:100C3000070605040100080A0B0C0D09080B000249
:100C40000202010009040000010202000005240064
:100C500010010524010101042402060524060001F7
:100C60000705810310004009040100020A0000008A
:100C7000070502024000000705830240000004034C
:100C800009042203410072006400750069006E00CF
:100C90006F0020004C0065006F006E006100720064
:100CA00064006F0018034100720064007500690061
:100CB0006E006F0020004C004C0043001201000247
:100CC00000000040412336800001010200011201B2
:100CD00000020200004041233680000101020001B1
:100CE00000C18081C105010902A1010901A100859E
:100CF00001050919012903150025019503750181D5
:100D0000029501750581030501093009310938157E
:100D100081257F750895038106C0C005010906A1DC
:100D2000018502050719E029E715002501750195E0
:100D3000088102950175088103950675081500253F
:100D4000650507190029658100C009040200010337
:100D5000000000092101010001226500070584034C
:100D600040000100000000000000002A2B280000C5
:100D70000000000000000000000000000000000073
:100D80000000002C9EB4A0A1A2A434A6A7A5AE3654
:100D90002D3738271E1F20212223242526B333B6C2
:100DA0002EB7B89F8485868788898A8B8C8D8E8F95
:100DB000909192939495969798999A9B9C9D2F3198
:100DC00030A3AD350405060708090A0B0C0D0E0FFC
:100DD000101112131415161718191A1B1C1DAFB178
:100DE000B0B500007E10B92B7430AF314C341124F3
:100DF0001FBECFEFDAE0DEBFCDBF14E0A0E0B1E070
:100E0000ECE3FCE602C005900D92A432B107D9F7DD
:100E100017E0A4E2B4E001C01D92A133B107E1F7ED
:100E20001DE0CEEEDDE004C02297FE010E94D63523
:100E3000C43ED107C9F70E94B9300C941C360C94FB
:100E40000000A0E0B0E0E7E2F7E00C94ED35EC0143
:100E5000A880B980CA80DB80A114B104C104D10488
:100E600041F484E2A82E89EDB82E8BE5C82E87E0E8
:100E7000D82EC601B5012DE133EF41E050E00E94CC
:100E8000A53527EA31E440E050E00E9451357B016E
:100E90008C01C601B5012DE133EF41E050E00E9425
:100EA000A535CA01B9012CEE34EF4FEF5FEF0E9478
:100EB00051356E0D7F1D801F911F97FF04C061503B
:100EC000704080409048688379838A839B839B012C
:100ED000AC015F77B901CA01CDB7DEB7EAE00C9487
:100EE00009360E942107089584E193E00E942107BA
:100EF00008956093140370931503809316039093E1
:100F000017030895A0E0B0E0E8E8F7E00C94E635B8
:100F1000EC012B016A016115710519F0FB01918348
:100F20008083C114D10449F0C6010297839728F049
:100F300020E030E040E050E0DCC0A9908A2D90E055
:100F40000E94DA35892BC9F7FDE2AF1621F4A9908A
:100F50003324339405C08BE2A81609F4A9903324F6
:100F6000C114D10421F0E0E1CE16D10411F5F0E373
:100F7000AF1669F48881883711F0883541F4A9806B
:100F8000229682E0382A20E1C22ED12C12C0C11450
:100F9000D10479F4E0E3AE1659F199E9E92E99E923
:100FA000F92E99E9092F99E1192F8AE0C82ED12C41
:100FB0003AC0FAE0CF16D10491F080E1C816D1040E
:100FC00029F0E8E0CE16D104F9F415C0BFEFEB2EFE
:100FD000BFEFFB2EBFEF0B2FBFE01B2F24C0A9E9F3
:100FE000EA2EA9E9FA2EA9E90A2FA9E11A2F1BC0B6
:100FF000F8E0CF2ED12CEFEFEE2EEFEFFE2EEFEF3D
:101000000E2FEFE11E2F0FC09601442737FD4095AC
:10101000542F6FEF7FEF8FEF9FEF0E948335C90151
:10102000DA017C018D0120E030E040E050E060E03A
:101030003601882477FC8094982C70EDB72EBA0C7A
:10104000F9E0FB1570F48A2D81548A3118F499EC7B
:10105000B92E06C08A2D81568A3148F589EAB82E04
:10106000BA0C8B2D90E08C159D050CF56F3FE9F0C7
:10107000E216F30604071507B8F0CA01B901A40186
:1010800093010E9451359B01AC018B2D90E0A0E0B3
:10109000B0E0280F391F4A1F5B1F281739074A077E
:1010A0005B0710F061E001C06FEFA990C6CF41145B
:1010B000510451F0662311F0219703C031FE04C0A2
:1010C0002297F201D183C08330FE07C0509540952E
:1010D000309521953F4F4F4F5F4F67FF0AC082E227
:1010E00090E09093300780932F072FEF3FEF4FEF63
:1010F0005FEFB901CA01CDB7DEB7E1E10C9402366A
:10110000FC0188279927E89421912032E9F32930BE
:1011100010F02E30C8F32B3241F02D3239F46894A0
:1011200004C00E94D508820F911D219120532A30BE
:10113000C0F31EF4909581959F4F089544E254E0CA
:101140000E94A3080895009731F4DA018D919C91D3
:10115000009709F40EC0DC01FB013D91219122238F
:1011600019F03217C9F3FACF332331F4DA011D92A3
:101170001C928827992708951197AF93BF93FB017D
:101180003D912191321771F4332321F48827992757
:10119000119702C01E921196FA01A193B0839F91FC
:1011A0008F910895222369F7EACF7AE0979F902DD7
:1011B000879F802D910D1124089580912604813000
:1011C00019F482E08093260480912604833019F478
:1011D00084E0809326040895009721F19C0140E06B
:1011E00050E068E478EE81E090E00E94A535C90106
:1011F000DA018F3F9105A105B10531F028F08FEF9D
:1012000090E0A0E0B0E008C00097A105B10521F48E
:1012100081E090E0A0E0B0E08093D1008091C00038
:10122000806103C08091C0008F7E8093C0000895CC
:10123000EBE6F0E0808180688083E8E6F0E0808182
:101240008160808308951F920F920FB60F92112430
:101250002F933F934F935F936F937F938F939F93BE
:10126000AF93BF93EF93FF931F9902C00E94DD08D5
:10127000FF91EF91BF91AF919F918F917F916F916E
:101280005F914F913F912F910F900FBE0F901F9044
:10129000189580915004E82FF0E03496DF0126E0A5
:1012A000AA0FBB1F2A95E1F720E030E040E050E0B4
:1012B00060E070E0F999FECFCB018A0F9B1F92BDD1
:1012C00081BDF89A80B5542F432F322F2227280F43
:1012D000311D411D511D6F5F7F4F6430710551F706
:1012E0002E513E4B414C5E4D19F020E030E01FC0C6
:1012F0009F0186E0220F331F8A95E1F72C5F3F4F55
:10130000E7E2F4E0F999FECF32BD21BDF89A80B54D
:1013100081932F5F3F4F84E0E035F80799F720E095
:1013200030E080912704893011F421E030E0C901D8
:10133000089589E08093270480E092ECA1E0B0E07A
:101340008093280490932904A0932A04B0932B043B
:1013500087E08093340480EC92E9ADEEB9E18093AC
:101360002C0490932D04A0932E04B0932F0485E0B9
:10137000809335048DEE9EEFADEABEED8093300490
:1013800090933104A0933204B0933304A6E3B4E005
:1013900080E090E0863010F0E0E004C0FC01E35112
:1013A000FC4FE081ED9301968831910599F782E039
:1013B00080934E048AE080934F040895843691050B
:1013C00020F4BC0180E090E025C08E3B910550F4F4
:1013D0008A559040BC0180E090E02AE030E040E097
:1013E00050E016C0823D910550F4845B9040BC01F2
:1013F00080E090E024E630E040E050E009C08D5C01
:101400009040BC0180E090E028E532E040E050E010
:101410000E94513524E630E040E050E00E94513512
:10142000089590E08C599F4F0E94DE090895DC01D9
:101430009896EC91F0E0E770F070EB51FC4F8081F2
:1014400008958F929F92AF92BF92CF92DF92EF92C8
:10145000FF920F931F938C010E94170AD801979651
:101460002C9130E043E150E0249FF001259FF00DE6
:10147000349FF00D1124E85EFC4F80809180A280A3
:10148000B38090E00F96AA2797FDA095BA2FBC01D4
:10149000CD0120E43FE14DE750E00E945135A50128
:1014A00094010E94833569017A0180ED97E0A0E004
:1014B000B0E0C80ED91EEA1EFB1ED80198968C918A
:1014C000887181F060E07EEE8AEB9BE0A5019401DB
:1014D0000E94833528513C4F4F4F5F4FC20ED31EA1
:1014E000E41EF51E87EE93E0A0E0B0E0C80ED91E22
:1014F000EA1EFB1EC701B60128EE33E040E050E0D3
:101500000E948335CA01B90128EE33E040E050E083
:101510000E9451351F910F91FF90EF90DF90CF9077
:10152000BF90AF909F908F9008958F3F910509F0E5
:1015300010F480E0089522E08030920710F481E0FA
:1015400008958050934010F083E0089582E008955C
:10155000CF92DF92FF920F931F93CF93DF93F82FD9
:10156000EB016A01182F1695E0E088819981D60178
:101570008C938A819B8111968C9311978C819D818C
:1015800012968C9312978E819F8113968C9313974A
:10159000288139814A815B816C817D818E819F8127
:1015A0009295990F990F907C832F8370982B852F9C
:1015B0008370880F880F982B872F83708295807F88
:1015C000982B14969C9385E090E0C80ED91E28961F
:1015D000EF5F1E1750F6F0FF21C0888199810E94AD
:1015E000950AF82E8A819B810E94950A182F8C817A
:1015F0009D810E94950A082F8E819F810E94950AE5
:10160000F294FF0CFF0C50ECF5221295107F1F296D
:10161000182B000F000F012BD6010C93DF91CF91F7
:101620001F910F91FF90DF90CF90089523E08032BB
:10163000920718F420E030E026C023E0883E9207AD
:1016400048F49C012F513340F4E036952795FA95E4
:10165000E1F719C027E0803D920720F49C012C5D42
:10166000334011C028E08839920718F02FEF33E09B
:101670000AC09C01285C3740E4E036952795EA953E
:10168000E1F72D503C4FC90108959C0136952795EF
:1016900025753575821B930B9C01369527953695DC
:1016A00027952373337383739373280F391FC901ED
:1016B00044E0969587954A95E1F7820F931F8F70C6
:1016C0009F7021E031E0AC01429FC001439F900D2B
:1016D000529F900D1124892F0895382F20E080917A
:1016E0001206909113068227932740E061E270E191
:1016F0009C01220F331F97FF04C0C901862797273B
:1017000001C0C9014F5F483099F790931306809349
:1017100012060895882339F0299800002A9A0000BB
:10172000299A00000895299800002A980000299A13
:1017300000000895299A000083B12998000090E0E4
:10174000F3E096958795FA95E1F7817008950F93E8
:101750001F93082F5E9A29985E9810E0802F80785A
:101760000E948A0B000F1F5F1830C1F729981F9144
:101770000F9108958F770E94A70B08950F931F93E1
:10178000082F10E0802F80780E948A0B000F1F5FC7
:101790001830C1F729981F910F9108950F931F9347
:1017A000299880E000E0182F110F0E949A0B810FFA
:1017B0000F5F0830C1F71F910F9108950E94BA0B77
:1017C0000E94CE0B5E9A08951F93162F80680E9488
:1017D000A70B812F0E94BE0B5E9A1F9108951F9345
:1017E000109130041827E7E2F4E0E80FF11D89E7D3
:1017F00067850E94E40B8DE3612F0E94E40B82E475
:10180000612F0E94E40B1F91089586E20E94DE0B77
:1018100008950F931F938C018CE1F80164810E945D
:10182000E40B8DE1F80165810E94E40B8EE1F80183
:1018300066810E94E40B80E2F80167810E94E40B5C
:1018400081E2F80160850E94E40B82E2F801618583
:101850000E94E40B83E2F80162850E94E40B84E2BB
:10186000F80163850E94E40B85E2F80164850E941B
:10187000E40B8AE2F80165850E94E40B8EE6F8012C
:1018800066850E94E40B8FE6F80167850E94E40BF1
:1018900080E7F80160890E94E40B81E7F801618923
:1018A0000E94E40B82E7F80162890E94E40B1F9119
:1018B0000F910895EF92FF920F931F93CF93DF93B1
:1018C0007B018C01603028E372072CE982072CE150
:1018D000920728F520E836E948E950E00E94833570
:1018E000E9016897B90180E090E020E839E647E631
:1018F0005FEF0E9451356E0D7F1D801F911F02E02A
:10190000660F771F881F991F0A95D1F721E732E0EC
:1019100040E050E00E948335890180E421C020E04E
:101920003DE241E351E00E948335E9016897B90146
:1019300080E090E020E033ED4EEC5EEF0E94513508
:101940006E0D7F1D801F911F660F771F881F991FC7
:1019500021E732E040E050E00E948335890180E6D3
:101960009E012F71622F680F85E70E94E40B86E7C6
:10197000612F0E94E40B87E7602F0E94E40BDF9148
:10198000CF911F910F91FF90EF9008959F92AF928A
:10199000BF92CF92DF920F93DF93CF9300D000D00E
:1019A000CDB7DEB7982E83E00E94DE0B80936C04E7
:1019B00084E00E94DE0B80936D0486E060E00E946C
:1019C000E40B87E061E00E94E40B89E06FE70E948E
:1019D000E40B8AE065E00E94E40B8BE065E10E9485
:1019E000E40B8CE062E10E94E40B8DE06DEF0E945D
:1019F000E40B8EE060E00E94E40B992019F087E789
:101A000093E008C080914E0423E1829FC00111241D
:101A1000885E9C4F0E94090C80E36CE80E94E40BF6
:101A200082E36FE00E94E40B83E362E40E94E40B34
:101A300084E36AE00E94E40B85E36AE20E94E40B1F
:101A400086E36DE20E94E40B87E364ED0E94E40B01
:101A500088E360E00E94E40B89E360E00E94E40B0D
:101A6000992049F02EE1A22E2EEBB22E21ECC22EAF
:101A70002EEDD22E08C0A0903004B0903104C0905A
:101A80003204D09033040AE38D2D9927AA27BB276F
:101A900089839A83AB83BC83802F69810E94E40B86
:101AA000802F8B5F69810E94E40BDC2CCB2CBA2C3D
:101AB000AA240F5F0E3341F783E46FEF0E94E40B1B
:101AC00084E46FEF0E94E40B85E46FEF0E94E40B67
:101AD00086E46FEF0E94E40B992019F08DE666E032
:101AE00003C08DE6609134040E94E40B89E760E056
:101AF0000E94E40B8AE7609135040E94E40B83E7BF
:101B000060E00E94E40B84E760E00E94E40B99200F
:101B100029F060EC72E98DEE99E108C060912C0427
:101B200070912D0480912E0490912F040E945A0CE4
:101B30000F900F900F900F90CF91DF910F91DF904A
:101B4000CF90BF90AF909F90089587E061E00E9492
:101B5000E40B8EE764E20E94E40B88E063E00E94FD
:101B6000E40B88E060E00E94E40B87E065E00E94FF
:101B7000E40B85E062E00E94E40B83E00E94DE0B50
:101B800080936C0484E00E94DE0B80936D040895C2
:101B9000582F40917D05842F90E0FC01EF70F0708C
:101BA0009F012F5F3F4F64E0959587956A95E1F718
:101BB0002817390751F0E359FA4F5083842F8F5F6C
:101BC0008F70407F842B80937D0508951F920F9224
:101BD0000FB60F9211241F932F933F934F935F9350
:101BE0006F937F938F939F93AF93BF93CF93DF9325
:101BF000EF93FF93C0918600D09187002091BF059D
:101C00003091C00580919E05882309F047C0CE0120
:101C1000821B930B9C0180914F0487FD02C0369577
:101C2000279599E0253C390708F18091AA03863071
:101C3000D0F08091AA038F3FB1F020E00EC0E22FD8
:101C4000F0E0EE0FFF1FDF01A156BA4F8D919C917E
:101C5000E657FC4F918380832F5F8091AA0328175A
:101C600070F310929D051092AA0318C082E02D3BDC
:101C7000380760F18091AA03803140F51091AA03E2
:101C8000C9010E94160BE12FF0E0EE0FFF1FE15695
:101C9000FA4F918380831F5F1093AA03D093C005EE
:101CA000C093BF05FF91EF91DF91CF91BF91AF91AD
:101CB0009F918F917F916F915F914F913F912F9164
:101CC0001F910F900FBE0F901F9018958FEF80936C
:101CD000AA03E4CF83E0809380008AE980938100A7
:101CE00080914F0486FD05C08091810080648093BF
:101CF00081008FEF9FEF90938900809388008091FF
:101D00006F00806280936F0008956F3020F0869599
:101D10008695805408958DE0689F802D1124089544
:101D2000982F80910B06882329F4933009F043C043
:101D300081E005C0813049F4913021F482E0809344
:101D40000B06089510920B060895803190F5E82F48
:101D5000F0E0E156FA4F90838F5F80930B0680315D
:101D600051F520919E05A1EAB5E0213039F4119694
:101D7000EC911197E695E6958C9109C08D919C9117
:101D80001197E92FE695E695E69596958795E031CA
:101D900040F4F0E090E0EE0FFF1FE657FC4F918318
:101DA000808310929D05129685E0AF3AB807E9F658
:101DB000089510920B0608950F931F93CF93DF930E
:101DC00090910B06992339F48F3009F002C181E01C
:101DD00080930B06FEC0983148F4E92FF0E0E256FC
:101DE000FA4F80839F5F90930B06F3C0983109F000
:101DF000EEC0882309F0EBC0C0E0D0E00BE010E0BB
:101E0000DE0163E0AA0FBB1F6A95E1F7C09FB00136
:101E1000C19F700DD09F700D1124FB01E156FA4F48
:101E200080812181922F977095958795FD01EE0F06
:101E3000FF1FE657FC4F91838083FB01E056FA4F6A
:101E400030813695369536952181422F4295440F43
:101E5000407E842F832B269526952695922F97706A
:101E600095958795FD01EE0FFF1FE457FC4F918379
:101E70008083FB01EF55FA4F808182958695869588
:101E800083704181942F990F990F292F282B429508
:101E900046954695437082818170880F880F382F50
:101EA000342B35952795FD01EE0FFF1FE257FC4FB0
:101EB00031832083FB01ED55FA4F30813695218126
:101EC000422F479544274795842F832B2695922FA1
:101ED000977095958795FD01EE0FFF1FE057FC4F1A
:101EE00091838083FB01EC55FA4F308132953F702E
:101EF0002181422F4295407F842F832B22952F7082
:101F0000922F977095958795FD01EE0FFF1FEE5666
:101F1000FC4F91838083FB01EB55FA4F8081881F32
:101F20008827881F4181942F990F292F282B441F20
:101F30004427441F82818370880F382F342B3595B6
:101F40002795FD01EE0FFF1FEC56FC4F31832083D8
:101F5000FB01E955FA4F3081369536952181422FA4
:101F60004295440F440F407C842F832B2695269561
:101F7000922F977095958795AA0FBB1FFD01EA5682
:101F8000FC4F9183808368557A4FFB012081229515
:101F9000269527704181342F330F330F330F832F52
:101FA000822B942F92959695977095958795A85624
:101FB000BC4F11969C938E932196C230D10509F0A7
:101FC0001FCF8091B50583FD02C010929D05109230
:101FD0000B06DF91CF911F910F910895DF92EF9241
:101FE000FF920F931F93CF93DF93682F40910B06BF
:101FF000442359F4883AB1F4109213061092120651
:1020000088EA0E946D0B81E06FC0413019F4809323
:10201000100604C0423031F480931106862F0E94CE
:102020006D0B5DC070911106272F30E0220F331F1A
:10203000E42FF0E0C90102968E179F0734F0433277
:1020400068F7E456FA4F6083E9CF2D5F3F4F409128
:10205000120650911306E217F30749F4962F80E019
:1020600048275927509313064093120638C0862FED
:1020700090E04817590789F580911006813069F57D
:10208000713118F080E180931106D0901106FFE9BC
:10209000EF2EF5E0FF2E00E010E01BC0F701D0812D
:1020A000C0E0818190E08C2B9D2BE3E09695879595
:1020B000EA95E1F70E94160BF801EE0FFF1FE657B5
:1020C000FC4F918380830F5F1F4F82E090E0E80E0A
:1020D000F91E0D1518F310929D0510920B068091B4
:1020E0000B06882319F08F5F80930B06DF91CF9149
:1020F0001F910F91FF90EF90DF900895109274045C
:10210000109279041092780410927B0410927A0451
:102110000895882319F460E071E002C063E071E083
:1021200081E696E00E946B2E0895CF92DF92EF92A7
:10213000FF921F93182F0E94DC299B01AC01809114
:102140000C0690910D06A0910E06B0910F06690144
:102150007A01C81AD90AEA0AFB0AD701C6018958C6
:102160009341A040B04010F010920B0620930C0653
:1021700030930D0640930E0650930F0690919E05E6
:10218000892F8150823020F4812F0E94900E0BC045
:10219000933021F4812F0E94DC0E05C0943019F495
:1021A000812F0E94EE0F1F91FF90EF90DF90CF9054
:1021B0000895FF920F931F93CF93DF93182F092F4A
:1021C000F62E8EE30E94E40B212F302FC901EC0183
:1021D00010E005C08FE769910E94E40B1F5F1F1597
:1021E000C8F385E064E00E94E40B83E00E94DE0B0C
:1021F00080936C0484E00E94DE0B80936D040E9447
:10220000DC2960936E0470936F0480937004909344
:10221000710487E069E00E94E40B81E0809326046A
:10222000DF91CF911F910F91FF9008950E94D910D7
:10223000809126048130D9F40E94DC2920916E041B
:1022400030916F044091700450917104621B730BC4
:10225000840B950B605A76488140904040F4E8CF5B
:1022600081E696E067E071E00E946B2E0895809110
:1022700026048130A9F3089587EF96E06EE70E9467
:1022800034300895BF92CF92DF92EF92FF920F9376
:102290001F93CF93DF936C0187EF96E06EE70E9468
:1022A0003430760100E010E0C0E0D0E080E2B82EEB
:1022B0000AC00830110521F49E012095F6012087FF
:1022C0000894E11CF11CF7016081862F8D57823044
:1022D00040F487EF96E06DE70E943430F7016081AB
:1022E0006B2587EF96E00E9434300115110551F0FF
:1022F000F70180819E01280F311DC32FDD27C20FFA
:10230000D31FD0700F5F1F4F0930110591F6DF9179
:10231000CF911F910F91FF90EF90DF90CF90BF90E2
:102320000895DF93CF93CDB7DEB729970FB6F89412
:10233000DEBF0FBECDBF382FE62F8091820590E023
:10234000019664E270E00E947035982F80938205B8
:1023500088E9898380E18A83913071F0913028F097
:10236000923099F09330E1F416C085E08B8381EFD1
:102370008C832F5F2D8317C09B8381EF8C8384E632
:10238000489FC00111249D830EC084E08B8381EFA0
:102390008C833D8308C09B8381EF8C83ED8303C0D6
:1023A0000E943C1104C0CE0101960E944211299660
:1023B0000FB6F894DEBF0FBECDBFCF91DF91089569
:1023C0000F931F93CF93DF93182F092F87EF96E07A
:1023D0006EE70E943430212F302FC901EC0110E04C
:1023E00000E288818D57823040F487EF96E06DE7F8
:1023F0000E94343088818027888387EF96E0699136
:102400000E9434301F5F193061F787EF96E06EE766
:102410000E943430DF91CF911F910F910895DF9387
:10242000CF93CDB7DEB729970FB6F894DEBF0FBEB6
:10243000CDBF382F80918205882379F48EEF898370
:102440003A836B83842F90E0959587958C832D83B9
:10245000198618861F821E822FC040917D05842F09
:1024600090E09C012F70307054E0959587955A95B7
:10247000E1F78217930721F18DEF89831A821B827E
:10248000DE01149620E008C0E359FA4F80818D9355
:10249000405F2F5F263069F0842F90E0FC0134E02C
:1024A000F595E7953A95E1F78F709070E817F90781
:1024B00059F740937D052A83CE0101960E94E011D1
:1024C0008091820590E0019666E070E00E94703590
:1024D0008093820529960FB6F894DEBF0FBECDBF5C
:1024E000CF91DF9108959F92AF92BF92CF92DF92EA
:1024F000EF92FF920F931F93B82EA62ED42EC22ECA
:10250000902E0E94DC297B018C0180916C0520912A
:102510007E0530917F05409180055091810588238B
:10252000B1F0D801C701821B930BA40BB50B815EE0
:102530009E42A040B04020F12C2DDC1408F42D2D3B
:102540008B2D6A2D422F292D0E94911111C0D80187
:10255000C701821B930BA40BB50B81539547A04079
:10256000B04070F08B2D6A2D4D2D2C2D0E940F1236
:10257000E0927E05F0927F0500938005109381051F
:102580001F910F91FF90EF90DF90CF90BF90AF9091
:102590009F900895219A229A23988BE060E00E94F0
:1025A0007E2A8CE061E00E947E2A089588E0809374
:1025B000C1008AE061E00E947E2A8AE060E00E9419
:1025C0000B2B0895AF92BF92CF92DF92EF92FF92C2
:1025D0000F931F93DF93CF93CDB7DEB76C970FB6F2
:1025E000F894DEBF0FBECDBF0E94DC297B018C01B9
:1025F00081E00E94C60CF4E7AF2E6E010894C11C66
:10260000D11CE3E0BE2EA982C60161E00E94161132
:10261000B09226040E94A50D6AEF70E080E090E081
:102620000E94022A80912604833009F08AC081E644
:1026300096E00E946F2B892B09F083C00E94DC2951
:102640006E197F09800B910B6058734C894C914037
:1026500008F077C0D8CF8FE70E94BA0B0E94CE0B4C
:10266000843509F05CC089830E94CE0B182F00E0EE
:1026700010936B0500936A050E94CE0B080F111D85
:1026800010936B0500936A050E94CE0B8093690539
:102690000E94CE0B80936805813108F040C0FF2472
:1026A00007C00E94CE0B085B1A4FF8018083F39499
:1026B0000F2D10E08091680590E0880F991F081792
:1026C000190778F380E78983CE01019661E00E94C3
:1026D000161183E0809326040E94A50D62E370E04A
:1026E00080E090E00E94022A809126048330A9F0C5
:1026F0008FE70E94BA0B0E94CE0B803581F489834C
:1027000001E514E00E94CE0BF80181938F01F4E003
:102710000C361F07B9F781E003C082E001C083E0F7
:102720006C960FB6F894DEBF0FBECDBFCF91DF9190
:102730001F910F91FF90EF90DF90CF90BF90AF90DF
:10274000089580912604833009F085CFE6CF83E099
:102750000E94DE0B80936C0484E00E94DE0B809369
:102760006D0487E061E00E94E40B6AE070E080E0C5
:1027700090E00E94022A0E94A50D000008950F9388
:102780001F93082F17C05F9A64E670E080E090E026
:102790000E94022A5F9864E670E080E090E00E9468
:1027A000022A1F5F101778F36CE271E080E090E07E
:1027B0000E94022A10E0F6CF482F392F25E00DC0E5
:1027C000F999FECF1FBA842F932F92BD81BD60BDB2
:1027D0000FB6F894FA9AF99A0FBE215059F0F99968
:1027E000FECF842F932F92BD81BDF89A80B56817D4
:1027F00039F7089582E00E94BF130895CF92DF92C7
:10280000EF92FF920F931F93CF93DF93C0E0D0E03E
:1028100008E110E08EE1C82E8EEBD82E81ECE82E78
:102820008EEDF82E8091500490E00496B6E0880F6B
:10283000991FBA95E1F7A7019601002E04C056959D
:102840004795379527950A94D2F78C0F9D1F622FD5
:102850000E94DC13219608501040C430D10511F7B6
:10286000C0E0D0E08091500490E0A6E0880F991F6E
:10287000AA95E1F78C5F9E4FFE01E95DFB4F8C0F3F
:102880009D1F60810E94DC132196C932D10551F74A
:10289000DF91CF911F910F91FF90EF90DF90CF903C
:1028A000089580E490E0609150040E94DC13089544
:1028B000F999FECF80E490E092BD81BDF89A80B591
:1028C00080935004843020F0109250040E945114E0
:1028D00008951F93182F0E94581480915004811757
:1028E00031F0143020F4109350040E9451141F91C1
:1028F00008951F93182F0E94DC2960937E05709322
:102900007F05809380059093810510936C051123BA
:1029100029F440E855E260E070E004C040E051EE88
:1029200060E070E087EF96E00E943A2F1F910895D3
:10293000809184058130D1F0813020F0823009F01F
:1029400043C037C082E10E943E2B892B09F03CC076
:1029500081E0809384050E94CE2960938505709361
:1029600086058093870590938805089582E10E94EB
:102970003E2B892BD9F40E94CE29209185053091D8
:1029800086054091870550918805621B730B840B67
:10299000950B695E734080409040B0F082E0809378
:1029A000840580ED97E00E94EC080895109284055C
:1029B000089582E10E943E2B892B31F080E090E067
:1029C0000E94EC08109284050895AF92BF92CF92B6
:1029D000DF92EF92FF920F931F93CF93DF938CE0E0
:1029E0000E94DE0B8823B9F581E696E063E171E091
:1029F0000E946B2E5F9A80E00E94C60C0E94A50D7B
:102A00005F9829C080919E05882339F087EF96E072
:102A10000E94FB2F0E9495101EC080910906C82FAE
:102A2000D0E09E012F5F3F4F2F71307080910806DC
:102A300090E02817390779F087EF96E00E94FB2F86
:102A4000C152DA4F88838091090690E001968F7118
:102A500090708093090687EF96E00E94C12F892B22
:102A600089F680912604843009F08CC00E94DC290C
:102A700060938D0570938E0580938F0590939005DC
:102A8000611571058105910561F481E090E0A0E098
:102A9000B0E080938D0590938E05A0938F05B09341
:102AA00090058091990590919A05816090939A057F
:102AB0008093990583E0809326048FE70E94BA0BE8
:102AC000C6EDD5E00E94CE0B899305E0CF3DD0073F
:102AD000C9F74091C1058091D605282F30E0842F99
:102AE00090E08227932786FF40C080E448274093E8
:102AF000C105C90188739070C89709F510E014C02A
:102B00001F5F80914F04E12FF0E084FF06C0EA527E
:102B1000FA4F80810E94C80D07C0EA52FA4F87EF32
:102B200096E060810E943430212F30E08091D605FC
:102B300090E0877090708217930714F716C02F7378
:102B40003070232B91F48091D7058093910580916B
:102B5000D805809393058091D90580939405809141
:102B6000DC0580939B0510929C0580910A068130BC
:102B700019F482E080930A0680910A06833011F4EA
:102B800010920A060E94DC295B016C018091950578
:102B900090919605A0919705B09198050097A10591
:102BA000B105C9F0A6019501281B390B4A0B5B0B37
:102BB000DA01C901885B9B40A040B04060F00E94F0
:102BC000050C80939205109295051092960510922F
:102BD00097051092980587E294E00E94210A2091BF
:102BE000890530918A0540918B0550918C058601AD
:102BF0007501E21AF30A040B150BE616F70608072F
:102C0000190708F4E9C0A0928905B0928A05C0921C
:102C10008B05D0928C0580919D05883008F0D4C03A
:102C200080919D058F5F80939D05E0908D05F090CC
:102C30008E0500918F0510919005E114F1040105B6
:102C4000110511F187E294E00E94210AAE18BF0835
:102C5000C00AD10A6A157B058C059D0588F4809110
:102C60004F0485FD04C080ED97E00E94EC081092AF
:102C70008D0510928E0510928F051092900504C05C
:102C800080E090E00E94EC089091C105907C9093C8
:102C9000C10500910906109108060117B1F1809154
:102CA0000A06823091F590589093C10587E294E02E
:102CB0000E94170A893010F048E002C0482F4150A6
:102CC00030E013C03F5FA32FB0E0812F90E0FC0104
:102CD000E152FA4F2081FD01EF53FA4F2083A150BA
:102CE000BA4F2C930196182F1F71341710F4101738
:102CF00049F710930806832F895C9091C105892BB1
:102D00008093C1053093FF051AC020910A06243034
:102D1000D1F49091FF05E0E0F6E0A2ECB5E0292FB8
:102D200030E02E0F3F1F02C081918D93E217F30711
:102D3000D9F7995C8091C105982B9093C10583E0E8
:102D400080930A0623C080918405823029F4916023
:102D50009093C1055F9A0FC09093C1055F9822239D
:102D600019F481E080930A0680910A06833019F4F1
:102D700084E080930A06F89480914F0487706AE893
:102D800073E042EC55E00E94A80A7894469A80913C
:102D900083050E94EF0B87E294E00E94170A682FD8
:102DA00081EC95E00E94D910E0918305EF5FE093FC
:102DB0008305E83131F0F0E0E95DFB4F878588233A
:102DC00059F41092830508C080919D05883009F45C
:102DD0005F9A89E080939D0580914F04887171F11D
:102DE00080912604823051F58091990590919A0541
:102DF000880F991F90939A058093990583E080939B
:102E000026040E94A50D0E94DC296093950570930D
:102E10009605809397059093980561157105810536
:102E2000910561F481E090E0A0E0B0E08093950529
:102E300090939605A0939705B093980580914F04C1
:102E400084FF1EC08091990590919A058E7F0E9403
:102E5000450B182F8091910560919B050E94850E6E
:102E6000082F80919205612F0E94850E282F809156
:102E7000930560919405402F009150040E947312B5
:102E800046980E949814DF91CF911F910F91FF9067
:102E9000EF90DF90CF90BF90AF90089510924605CD
:102EA00085E6E1EEF4E0DF011D928A95E9F70895E9
:102EB000FF920F931F938C01F62E81E696E00E94FD
:102EC000D02BF80184818F2584831F910F91FF906F
:102ED0000895FF920F931F938C01F72E0E945817AD
:102EE000C8016F2D0E9458171F910F91FF900895F0
:102EF000BF92CF92DF92EF92FF920F931F937C01CC
:102F0000B62E6A0101E616E0C80165EB0E94D02BDF
:102F1000C80162E60E94D02BF7011482C7016B2D15
:102F20000E945817C701B6010E9469171F910F919F
:102F3000FF90EF90DF90CF90BF9008951F93182FD0
:102F40008F3711F08830E1F5E0914605EE2309F462
:102F500055C0E150E0934605F0E0EF51FB4F108281
:102F600081E696E06DE00E94D02B10E00AC0E12FD0
:102F7000F0E0EF51FB4F81E696E060810E94D02B9C
:102F80001F5F80914605181790F381E696E060E296
:102F90000E94D02B81E696E06DE00E94D02B10E0DD
:102FA0000AC0E12FF0E0EF51FB4F81E696E060812F
:102FB0000E94D02B1F5F80914605181790F31CC00C
:102FC0008B3119F40E944E171FC08D30E9F08A3002
:102FD000D9F080914605843688F481E696E0612F29
:102FE0000E94D02B80914605E82FF0E0EF51FB4F77
:102FF00010838F5F8093460580E007C081E696E0EE
:1030000067E00E94D12CF8CF81E01F9108951F93B3
:10301000CF93DF93C6E3D4E010E03BC081E696E0B7
:1030200062E271E00E94682E81E696E0612F4AE03C
:1030300050E00E94DF2D81E696E06FE271E00E9491
:10304000682E699170E080E090E02091350430E0D6
:1030500040E050E00E94513520E137E240E050E08E
:103060000E945135DC01CB0140912C0450912D047C
:1030700060912E0470912F04480F591F6A1F7B1F07
:1030800081E696E02AE030E00E94A62D1F5F18310D
:1030900019F08881882311F6DF91CF911F9108954F
:1030A000EF92FF920F931F93882339F481E696E005
:1030B0006CE47AE00E94EF2C3BC090E00E94DE09B5
:1030C00024E630E040E050E00E948335122F032FC9
:1030D000F42EE52E622F732F842F952F2AE030E0F7
:1030E00040E050E00E94833581E696E0BA01A901F4
:1030F0002AE030E00E94972D81E696E06EE20E9481
:10310000D12C612F702F8F2D9E2D2AE030E040E0D2
:1031100050E00E948335AB01BC0181E696E02AE0D5
:1031200030E00E94972D81E696E063E70E94032D30
:103130001F910F91FF90EF900895FF920F931F93AF
:10314000CF93DF9381E696E062E47AE00E94AE2CB2
:1031500080915104813041F481E696E069E27AE0A1
:103160000E94EF2CFF2466C0823029F481E696E0AD
:1031700062E17AE0F5CF8430A9F781E696E06EEF60
:1031800079E0EECFCF2DD0E0C930D1051CF06F2D06
:10319000685C02C06F2D6F5C81E696E00E94D12CC6
:1031A00081E696E066EF79E00E94AE2CBE016F5F8B
:1031B0007F4F81E696E04AE050E00E94412E81E692
:1031C00096E06BEE79E00E94AE2C8E010F5A1B4FF9
:1031D000D8011196EC91E032F8F481E696E06EEDBC
:1031E00079E00E94AE2CF8018181803130F081E6D7
:1031F00096E063E371E00E94682ECF5ADB4F69814D
:1032000070E06F7070706F5F7F4F81E696E04AE00C
:1032100050E00E94542E0DC0F0E0EF70F070EE0F01
:10322000FF1FEB54FC4F6081718181E696E00E94A4
:103230006B2EF39480916905F81608F4A3CF81E60C
:1032400096E063EC79E00E94AE2C809169040E94C4
:10325000501881E696E068EA79E00E94AE2C8091F1
:103260006A040E94501881E696E06DE879E00E94B9
:10327000AE2C80916B040E94501881E696E062E7C4
:1032800079E00E94AE2C40916104509162046091FB
:10329000630470916404411551056105710539F1AC
:1032A00081E696E02AE030E00E94A62D81E696E0D5
:1032B0006FE379E00E94AE2C809165040E94110AB0
:1032C000AB01BC0181E696E02AE030E00E94A62D29
:1032D00081E696E06BE179E00E94AE2C81E696E013
:1032E000609166044AE050E00E94F12D06C081E63C
:1032F00096E062E179E00E94EF2C81E696E065EFCE
:1033000078E00E94AE2C609167047091680481E6B9
:1033100096E04AE050E00E94CB2D81E696E068ED11
:1033200078E00E94AE2C60916004603150F470E04F
:103330006F5F7F4F81E696E04AE050E00E94542E96
:1033400006C081E696E06FEC78E00E94EF2C81E603
:1033500096E062EB78E00E94AE2C80915F0480FDE5
:1033600003C065E371E002C069E371E081E696E0C5
:103370000E946B2E81E696E065E978E00E94AE2C13
:1033800080915F0482700E94891081E696E066E772
:1033900078E00E94AE2C80915F0484700E948910B6
:1033A00081E696E067E578E00E94AE2C80915F04AC
:1033B00088700E948910DF91CF911F910F91FF902B
:1033C00008951F93CF93DF9381E696E066E97BE053
:1033D0000E94AE2C40912C0450912D0460912E043B
:1033E00070912F0481E696E02AE030E00E94A62D3D
:1033F00081E696E060E87BE00E94AE2C40913004CC
:1034000050913104609132047091330481E696E06A
:1034100020E130E00E94A62D81E696E06AE67BE09E
:103420000E94AE2C81E696E0609134044AE050E0C0
:103430000E94F12D81E696E064E57BE00E94AE2CCF
:1034400081E696E0609135044AE050E00E94F12D5B
:1034500081E696E06EE37BE00E94AE2CC6E3D4E00A
:1034600010E012C0112331F081E696E06DE371E0C7
:103470000E94682E81E696E069914AE050E00E9441
:10348000DF2D1F5F183119F08881882359F781E6F5
:1034900096E00E94D92C81E696E068E27BE00E94EB
:1034A000AE2C81E696E060914E044AE050E00E9426
:1034B000F12D81E696E063E17BE00E94AE2CE09185
:1034C0004F04F0E0E770F070EE0FFF1FEB52FC4F7F
:1034D0006081718181E696E00E946B2E81E696E024
:1034E0006EEF7AE00E94AE2C80914F0490E08871DC
:1034F00090708830910589F0893091051CF4892BF2
:1035000039F01BC08031910569F04897B1F40FC0C4
:1035100081E696E065EF7AE00EC081E696E069EE1E
:103520007AE009C081E696E063EE7AE004C081E6C5
:1035300096E069ED7AE00E94EF2C81E696E065EC7A
:103540007AE00E94AE2C40912804509129046091A9
:103550002A0470912B0481E696E02AE030E00E9474
:10356000A62D81E696E06CEA7AE00E94AE2C80916E
:103570004F0480720E94891081E696E063E97AE048
:103580000E94AE2C80914F0480740E94891081E6C5
:1035900096E06AE77AE00E94AE2C80914F04807832
:1035A0000E94891081E696E06DE57AE00E94AE2CDB
:1035B00087E294E00E94210AAB01BC0181E696E01B
:1035C0002AE030E00E94972D81E696E068E57AE0F7
:1035D0000E94AE2C87E294E00E94210A9B01AC017C
:1035E00060E472E48FE090E00E94833581E696E02B
:1035F000BA01A9012AE030E00E94972D81E696E009
:1036000065E57AE00E94EF2CDF91CF911F9108953C
:10361000EF92FF920F931F937C0101E616E0C80121
:103620006F2D70E04AE050E00E94BA2DC8016EE2B2
:103630000E94D12CB70154E0769567955A95E1F731
:103640006F707070C8014AE050E00E94BA2DC80146
:103650006EE20E94D12C8FE0E822FF24C801B7015E
:103660004AE050E00E94BA2D1F910F91FF90EF9019
:1036700008950F931F93CF93DF932091E0042F3F82
:10368000A9F581E696E067ED75E00E94AE2C84E531
:1036900093E00E94081B81E696E066EB75E00E94CD
:1036A000AE2C80916A0590916B050E94081B81E603
:1036B00096E063E875E00E94EF2C81E696E060E614
:1036C00075E00E94EF2C81E696E068E475E00E94C8
:1036D000EF2C81E696E063E275E00E94EF2C81E634
:1036E00096E00E94D92C0E949D1869C012160CF019
:1036F00066C0332727FD30958091690590E08217D9
:1037000093070CF45CC081E696E06EE075E00E94E1
:10371000AE2C6091E004772767FD709581E696E016
:103720004AE050E00E94542E81E696E063EE74E099
:103730000E94AE2C08E210E03AC0C12FD0E0CC0FBE
:10374000DD1FC85BDA4F288130E08091E0049927C3
:1037500087FD909501972817390741F581E696E096
:103760006FE371E00E94682E81E696E0602F4AE0E8
:1037700050E00E94DF2D81E696E063E471E00E9454
:10378000682EE981F0E0EF70F070EE0FFF1FEB5450
:10379000FC4F6081718181E696E00E94682E81E68F
:1037A00096E067E471E00E94682E0F5F1F5F8091D2
:1037B0006805181710F281E696E00E94D92CDF9177
:1037C000CF911F910F910895CF92DF92EF92FF92C8
:1037D0000F931F93DF93CF93CDB7DEB76C970FB6E0
:1037E000F894DEBF0FBECDBF282F8091E0048F3F3D
:1037F00009F050C1822F992787FD9095A92FB92FE5
:10380000FC013A97EF36F10508F03DC1EA5AFF4F47
:10381000EE0FFF1F0590F491E02D099481E696E0EC
:1038200069E471E0B4C081E696E069E471E00E9469
:103830006B2E22C181E696E065E571E00E946B2E59
:1038400085E78983DE011296E1E5F4E08BE10190E2
:103850000D928150E1F7CE0101966CE10E941611A4
:103860000E94A50D83E08093260468EC70E080E060
:1038700090E00E94022A80912604843009F003C15E
:103880008FE70E94BA0B0E94CE0B8983853509F021
:10389000FAC081E696E065EC74E00E94EF2C81E6C8
:1038A00096E067EA74E00E94EF2C81E696E069E812
:1038B00074E0B2C081E696E06DE671E00E946B2E86
:1038C00089E68983CE01019661E00E9416110E946B
:1038D000A50D83E08093260468EC70E080E090E022
:1038E0000E94022A80912604843009F0CCC08FE720
:1038F0000E94BA0B0E94CE0B89838E010E5F1F4F70
:10390000BDE1EB2EF12CEC0EFD1E0E94CE0BD8017A
:103910008D938D01AE15BF05C1F7A1E5B4E0FE01A1
:1039200032968BE101900D928150E1F789818934C3
:1039300009F0A9C081E696E06BE674E00E94EF2CE6
:1039400081E696E06DE474E00E94EF2C81E696E05B
:103950006FE274E061C081E696E067E871E00E9482
:103960006B2E8EEF8093E0048EC020522750422FA2
:103970004053242F332727FD30958091690590E02F
:10398000821793073CF481E696E066E971E00E94B5
:103990006B2E79C04093E0046FC084E18093E00413
:1039A00081E696E068EF73E037C085E18093E0043C
:1039B00081E696E061EC73E02FC086E18093E0043D
:1039C00081E696E06AE873E027C087E18093E0042F
:1039D00081E696E060E473E01FC088E18093E00434
:1039E00081E696E06FE273E017C089E18093E0041E
:1039F00081E696E06BE173E00FC08AE18093E0041A
:103A000081E696E066E073E007C08BE18093E00416
:103A100081E696E06EED72E00E94EF2C34C081E604
:103A200096E064EC72E00E94EF2C80915F0491E0DC
:103A30001DC081E696E06EEA72E00E94EF2C809154
:103A40005F0492E013C081E696E069E972E00E94AB
:103A5000EF2C80915F0494E009C081E696E06EE768
:103A600072E00E94EF2C80915F0498E08927809398
:103A70005F048FEF8093E0040E94391B04C081E64D
:103A800096E00E94962B81E696E00E946F2B892B90
:103A9000B1F776C1822F0E949E17882309F470C166
:103AA00080914605882321F48FEF8093E00460C164
:103AB00081EE94E060E070E040E050E00E94820718
:103AC0009B01AC019091E004963109F47CC09731E0
:103AD00064F4943109F463C095310CF06AC0892F05
:103AE00081508D3008F034C113C0993109F4E5C01C
:103AF0009A313CF4973109F470C0983109F028C12B
:103B0000D2C09A3109F4E7C09B3109F021C1F4C059
:103B1000E92FFF27E7FDF0958091690590E08E176A
:103B20009F070CF415C1DA01C9010197A109B10978
:103B30008097A105B10548F010E0A8E2FA2E00E058
:103B40006F010894C108D10825C0EF5AFB4F822F9E
:103B500081508083E5C0612F70E0660F771F685B3E
:103B60007A4FFB01808190E08C159D0591F48F2D9B
:103B700090E0A0E0B0E082179307A407B50741F4F6
:103B8000F601EF5AFB4FDB0111968C91818301E026
:103B9000F3941F5F809168051817E8F2BFC02F3FAC
:103BA00031054105510511F008F0D2C02093690498
:103BB000B7C02F3F31054105510511F008F0C8C0CD
:103BC00020936A04ADC02F3F31054105510511F026
:103BD00008F0BEC020936B04A3C08091E104806212
:103BE000803719F582EE94E060E070E040E050E04C
:103BF0000E9482079B01AC01DC01CB010197A10966
:103C0000B1090897A105B10508F0B5C0CA01B9010D
:103C100024ED30E340E050E00E9451359B01AC01BF
:103C20002A5E3C4A4A46554E24C0863611F582EE3D
:103C300094E060E070E040E050E00E9482079B0169
:103C4000AC01DC01CB010197A109B1090797A105DE
:103C5000B10508F090C0CA01B90128EA31E640E098
:103C600050E00E9451359B01AC01245E3C434E461E
:103C7000544E211531054105510561F0DA01C901A4
:103C80008054914EAD49B8418158904FAA4FB240EF
:103C900008F05EC020936104309362044093630493
:103CA000509364043DC02F3F31054105510511F08B
:103CB00008F04EC02093650433C0DA01C9010197B2
:103CC000A109B1098F3F9105A105B10508F040C0D8
:103CD0002093660425C0DA01C901845C9940A040A4
:103CE000B0408D549D41A040B04030F43093680402
:103CF0002093670401E001C000E021153105410572
:103D0000510511F48FEF07C02131310541055105EF
:103D100028F4822F81508093600402C00023C1F0F8
:103D2000809147058823D1F480913004909131042B
:103D3000A0913204B09133040196A11DB11D80936E
:103D4000300490933104A0933204B093330406C03E
:103D500081E696E068EA71E00E946B2E0E944E17A1
:103D60008FEF8093E00481E696E06AE00E94032DE5
:103D70000E94391B05C021E030E040E050E07ECFDA
:103D80006C960FB6F894DEBF0FBECDBFCF91DF911A
:103D90001F910F91FF90EF90DF90CF90089581E6F3
:103DA00096E062E372E00E94EF2C81E696E06AE121
:103DB00072E00E94EF2C81E696E00E946F2B892B27
:103DC00031F081E696E00E94962B0E94E41B0E944F
:103DD000E212823019F0833069F405C081E696E082
:103DE0006CEF71E004C081E696E065EE71E00E9440
:103DF000EF2C08958FEF8093E004109247050E9406
:103E0000391B0CC081E696E00E946F2B892B31F0A4
:103E100081E696E00E94962B0E94E41B8091E004CC
:103E20008E3F81F708958091E004843009F46FC0DB
:103E3000853084F4813009F45BC0823024F48F3FF4
:103E400009F085C014C0823009F457C0833009F0EE
:103E50007EC058C0863009F464C086300CF45CC063
:103E6000873009F463C0893009F071C06AC081E607
:103E700096E06AE478E00E94EF2C84E593E00E94EB
:103E8000081B81E696E062E378E00E94EF2C81E671
:103E900096E06DE078E00E94EF2C81E696E063EE1C
:103EA00077E00E94EF2C81E696E062EC77E00E94DA
:103EB000EF2C81E696E065E977E00E94EF2C81E641
:103EC00096E06FE677E00E94EF2C81E696E06BE4E7
:103ED00077E00E94EF2C81E696E064E277E00E94B2
:103EE000EF2C81E696E00E94D92C0E94E1192FC0A8
:103EF00081E696E067E077E028C081E696E062EE32
:103F000076E023C081E696E06DEC76E01EC081E6A7
:103F100096E06EEA76E019C081E696E06AE676E021
:103F200014C081E696E065E576E00FC081E696E094
:103F300060E476E00E94EF2C81E696E06AEF75E09F
:103F400004C081E696E064EE75E00E94EF2C6AE022
:103F500070E080E090E00E94022A04C081E696E0D2
:103F60000E94962B81E696E00E946F2B892BB1F779
:103F700008952F923F924F925F926F927F928F920D
:103F80009F92AF92BF92CF92DF92EF92FF920F93E8
:103F9000DF93CF93CDB7DEB7A8970FB6F894DEBF07
:103FA0000FBECDBF7E010894E11CF11C80E1D7015A
:103FB0001D928A95E9F781E696E066EC71E00E9431
:103FC0006B2E0E94A71320E431EE4DE958E129A39E
:103FD0003AA34BA35CA380EC91EDA8E9BBE18D8FE4
:103FE0009E8FAF8FB8A324EF31E040E050E0298FDF
:103FF0003A8F4B8F5C8F20E5822E23EC922EA12CE2
:10400000B12C80E491EEADE9B8E18D8B9E8BAF8B46
:10401000B88F44245524320100E022243324198A25
:104020001A8A1B8A1C8A0DC181E696E00E94962B93
:104030008434C9F0853434F48332C9F18C3209F008
:10404000CEC046C0833509F0CAC029A13AA14BA110
:104050005CA1C901DA018D8B9E8BAF8BB88F442494
:1040600055243201EEC081E696E064E40E94D12C32
:1040700081E696E040E451EE6DE978E12AE030E037
:104080000E94052E81E696E06CE20E94D12C81E62A
:1040900096E040EC51ED68E97BE12AE030E00E94D7
:1040A000052E81E696E06CE20E94032DCAC01982BB
:1040B0001A821B821C821D821E821F82188619860C
:1040C0001A861B861C861D861E861F86188A3CC083
:1040D0000F5F043009F0B5C069817A818B819C81C2
:1040E00028EE33E040E050E00E94513569A37AA306
:1040F0008BA39CA36D817E818F8198850E94513511
:104100006D8F7E8F8F8F98A329853A854B855C852F
:10411000298F3A8F4B8F5C8F6D857E858F8598892F
:1041200028EE33E040E050E00E9451354B015C0145
:1041300060323EE4730730E0830730E0930730F4E9
:104140008CE162E30E94E40B00E07BC0603345E752
:10415000740740E0840740E0940718F48CE162E2C1
:10416000F1CF60345CE9750750E0850750E09507B2
:1041700018F48CE166E2E6CF80E5881683EC9806B9
:1041800080E0A80680E0B80618F48CE162E1DACF9E
:1041900090E689169AEE990690E0A90690E0B90695
:1041A00018F48CE165E1CECFA0E78A16A1E19A066A
:1041B000A1E0AA06A0E0BA0618F48CE161E0C2CF43
:1041C000B0EA8B16B6E89B06B1E0AB06B0E0BB06E2
:1041D00018F48CE163E0B6CF8CE165E0B3CF805397
:1041E0008A3078F5C02EDD24CC0CDD1CCC0CDD1C17
:1041F000E1E0F0E0EC0FFD1FCE0EDF1E282F33278D
:1042000027FD3095432F532F2DA33EA34FA358A72F
:10421000D6016D917D918D919C912AE030E040E036
:1042200050E00E9451352DA13EA14FA158A5260F67
:10423000371F481F591FD6012D933D934D935C9313
:10424000139781E696E00E946F2B892B09F0ECCE44
:10425000411451046104710499F46D897E898F8938
:10426000988D0E945A0C61E070E080E090E00E941E
:10427000022A22242A943324198A1A8A1B8A1C8A25
:10428000298D3A8D4B8D5C8D42165306640675065A
:10429000D0F40E94050C29893A894B895C89280F42
:1042A000311D411D511D298B3A8B4B8B5C8B381670
:1042B00008F4382E821508F4282E0894411C511C4D
:1042C000611C711C64C06D897E898F89988D28EE70
:1042D00033E040E050E00E94833581E696E0BA0189
:1042E000A9012AE030E00E94972D81E696E06CE279
:1042F0000E94D12C81E696E0632D4AE050E00E94B6
:10430000DF2D81E696E06CE20E94D12C69897A89E2
:104310008B899C89A30192010E94833581E696E0F6
:10432000BA01A9012AE030E00E94972D81E696E0CB
:104330006CE20E94D12C81E696E0622D4AE050E0CA
:104340000E94DF2D81E696E06CE20E94032D8D89AC
:104350009E89AF89B88D880D991DAA1DBB1D8D8BB7
:104360009E8BAF8BB88F2D8D3E8D4F8D58A128170A
:1043700039074A075B0740F489A19AA1ABA1BCA108
:104380008D8B9E8BAF8BB88F44245524320129A18D
:104390003AA14BA15CA1285E33404040504009F057
:1043A00050CFA8960FB6F894DEBF0FBECDBFCF9109
:1043B000DF910F91FF90EF90DF90CF90BF90AF9083
:1043C0009F908F907F906F905F904F903F902F9035
:1043D0000895CF92DF92EF92FF920F931F93DF9396
:1043E000CF93CDB7DEB7E8970FB6F894DEBF0FBE18
:1043F000CDBF7C01FC018281883009F4ABC08930DB
:10440000A8F4843009F45FC0853048F48230E9F1C3
:10441000833008F04DC0813009F080C123C0863060
:1044200009F482C0873008F08BC060C0883609F478
:10443000D4C0893650F4863609F4AFC0873608F008
:10444000C5C0853609F06AC18FC08A3609F4FEC03E
:104450008A3608F4F2C08B3609F438C1873C09F07B
:104460005DC149C1C70161E049E250E00E9478178F
:1044700007E214E0C701F80161918F010E9458170B
:10448000F4E000351F07B1F753C1C70162E04BE10B
:1044900050E00E94781701E514E0C701F80161912E
:1044A0008F010E945817F4E00C361F07B1F740C186
:1044B000C70163E041E050E00E9478170E94E212D9
:1044C000682FC70133C1C70164E041E050E00E949A
:1044D0007817C70161E00E94581781E696E0F7015E
:1044E00064810E94D02B0E94B91F28C140916805A9
:1044F00050E0440F551FC70165E00E94781700E0A7
:1045000010E009C0F801E85BFA4FC70160810E9422
:1045100058170F5F1F4F8091680590E0880F991F13
:104520000817190778F304C1C70166E042E050E0BC
:104530000E947817C70164E573E00E946917F8C00C
:10454000C70167E041E050E00E947817C701609121
:104550006905ECC0C70168E041E050E00E947817AF
:10456000C70160915004E2C0C70165E641E050E038
:104570000E947817F70187819085899709F0D4C048
:10458000D701E7E2F4E019968C911997819311967F
:1045900084E0E035F807B9F7ABC0C70166E641E053
:1045A00050E00E947817F701878190854B9709F0BA
:1045B000BBC0D701E1E5F4E019968C91199781937E
:1045C000119684E0EC36F807B9F792C0C70167E6A8
:1045D00041E050E00E94781789C0C70168E641E0D9
:1045E00050E00E94781785E78983DE011296E1E5A5
:1045F000F4E08BE101900D928150E1F7CE0101963C
:104600006CE10E9416110E94A50D83E080932604A0
:1046100068EC70E080E090E00E94022A809126041D
:10462000843009F081C08FE70E94BA0B0E94CE0B44
:104630008983853509F078C05BC0C70169E641E030
:1046400050E00E9478170E94990952C0C7016AE69B
:1046500041E050E00E94781789E68D8FCE014D969B
:1046600061E00E9416110E94A50D83E0809326044C
:1046700068EC70E080E090E00E94022A80912604BD
:10468000843009F051C08FE70E94BA0B0E94CE0B14
:104690008D8F8E01025E1F4F39E3C32ED12CCC0EBD
:1046A000DD1E0E94CE0BF80181938F01EC15FD05F4
:1046B000C1F7A1E5B4E0FE017E968BE101900D9279
:1046C0008150E1F78D8D893479F512C0C7016BE611
:1046D00041E050E00E947817F70181850E9469143B
:1046E0000E944909892B21F40E9499090E94FE1316
:1046F000C70161E01BC0C70167EC41E050E00E94C8
:104700007817C70161E00E94581781E696E0F7012B
:1047100064810E94D02B1092720410C0C7016AEC11
:1047200041E050E00E947817C70160E00E945817EE
:1047300081E696E0F70164810E94D02BE8960FB6DF
:10474000F894DEBF0FBECDBFCF91DF911F910F91C7
:10475000FF90EF90DF90CF9008956F927F928F92AD
:104760009F92AF92BF92CF92DF92EF92FF920F9300
:104770001F93CF93DF9381E08093720488E7E82E44
:1047800084E0F82E04E0C02ED12CCE0CDF1C14E601
:10479000612EB4E07B2EA6E09A2EF5E08F2EE2E0AB
:1047A000AE2E73E0B72EB8C081E696E00E946F2B64
:1047B000892B09F4B1C0A9C081E696E00E94962B2E
:1047C000982F8093730480917404833021F1843096
:1047D00028F4813099F08230B8F409C0853009F4AA
:1047E00050C0853020F1863009F08FC067C0953BFE
:1047F00009F08BC081E08093740487C0923609F081
:1048000082C0A092740481C0909375049093760442
:10481000B09274047AC090937804F7011182809169
:104820007604892780937604709274046EC0D92F21
:10483000C0E020917804309179042C2B3D2B3093EB
:1048400079042093780480917604892780937604F4
:10485000809274042536310508F457C083E794E04C
:104860006CEC41E050E00E94781783E794E061E04F
:104870000E94581781E696E0609177040E94D02B41
:1048800042C020917A0430917B04F901ED58FB4F2E
:104890009187809176048927809376042F5F3F4F1C
:1048A00030937B0420937A0480917804909179046A
:1048B0002817390750F19092740427C000917604AC
:1048C000091729F483E794E00E94E92113C01091AD
:1048D000750483E794E06BEC42E050E00E947817A7
:1048E00083E794E0612F0E94581783E794E0602FDC
:1048F0000E945817F601862D11928A95E9F71092B9
:104900007B0410927A041092740481E696E00E946F
:104910006F2B892B09F050CF80917204813009F4FC
:1049200043CFDF91CF911F910F91FF90EF90DF90D8
:10493000CF90BF90AF909F908F907F906F90089591
:10494000DF92EF92FF920F931F93CF93DF930E941A
:10495000DC296115710581059105C9F30E9479076C
:1049600010923004109231041092320410923304E9
:10497000DD24E0903004F090310400913204109175
:104980003304102F0F2DFE2CEE240E9474072FEFFE
:1049900030E040E050E00E94A535E60EF71E081F0B
:1049A000191FE0923004F092310400933204109306
:1049B0003304D39484E0D816E1F6C6E3D4E010E0E3
:1049C00017C00E94740722E330E040E050E00E94EC
:1049D000A5356F5FE6E3F4E090E004C081918617AF
:1049E00081F39F5F9117D0F369931F5F183119F01E
:1049F0008881882331F7DF91CF911F910F91FF902C
:104A0000EF90DF9008951F931091E0041F3F09F08D
:104A1000BFC0893409F466C08A342CF5883309F4A0
:104A200076C089336CF4803309F481C081330CF093
:104A30006CC08B3109F44CC0813209F0A3C03CC07A
:104A4000813409F483C082343CF4893309F46DC0A5
:104A5000803409F097C030C0823409F482C08634B3
:104A600009F090C04FC0823609F47BC083368CF4C5
:104A7000883571F1893534F48235E9F1833509F0EF
:104A800081C01FC08A3509F478C0813609F07AC028
:104A90005DC0823781F1833734F4863699F18936E7
:104AA00009F070C01FC0883799F08A3709F465C0D3
:104AB000833709F067C005C081E696E069E471E0DC
:104AC00017C00E94FE1381E696E063ED71E006C018
:104AD0000E94490981E696E06DEE71E00E946B2E1E
:104AE0008EEF4EC00E94990981E696E06CE072E07C
:104AF0000E946B2E47C00E94A02481E696E065E2EA
:104B000072E0F6CF0E9407183DC0805339C081E69D
:104B100096E062ED71E00E94EF2C90914F04892F96
:104B2000885F8871977E892B0CC089E029C081E657
:104B300096E06FEB71E00E94EF2C80914F0490E2C1
:104B4000892780934F041093E0041CC081E696E00F
:104B500069EA71E00E94EF2C80914F0490E489276C
:104B600009C081E696E068E971E00E94EF2C80912F
:104B70004F04805880934F0402C00E94CF1E8FEFD5
:104B80008093E0048091E0048E3F09F4E8C0DFC028
:104B90000E949E17882309F4E2C08091460588236D
:104BA00021F48FEF8093E004D2C081EE94E060E0C6
:104BB00070E040E050E00E9482079B01AC018091D0
:104BC000E004843009F441C0853044F4823041F17E
:104BD000833094F5813009F096C00DC0863009F419
:104BE00067C086300CF43EC0873009F469C0893054
:104BF00009F089C075C0DA01C9018154914EAD49EF
:104C0000B8418F57904FAA4FB24008F07CC0209314
:104C10002C0430932D0440932E0450932F049AC0FB
:104C20002093300430933104409332045093330482
:104C300081E0809347058EC028303105410551053C
:104C400008F061C02093340485C0DA01C9010197DE
:104C5000A109B1090A97A105B10508F054C0209334
:104C6000350478C081EE94E06DE371E00E949E0807
:104C700010E00EC0183130F4E12FF0E0E95DFB4F99
:104C800087871F5F80E090E06DE371E00E949E08DF
:104C9000009759F00E948008009761F706C0E12F45
:104CA000F0E0E95DFB4F17861F5F1831C0F352C07B
:104CB000253031054105510530F520934E044AC099
:104CC000DA01C9010197A109B1090697A105B1054A
:104CD000D0F480914F04887F822B80934F043AC098
:104CE000DA01C9010197A109B1098050924CA14094
:104CF000B04048F4209328043093290440932A04B8
:104D000050932B0427C081E696E068EA71E00E9488
:104D10006B2E13C08091300490913104A091320425
:104D2000B09133040196A11DB11D8093300490937E
:104D30003104A0933204B09333040E944E178FEFD6
:104D40008093E00481E696E06AE00E94032D0E94D1
:104D5000131F05C0809147058823E1F2EECF1F9114
:104D600008958FEF8093E004109247050E94131F6F
:104D70000CC081E696E00E946F2B892B31F081E612
:104D800096E00E94962B0E9403258091E0048E3FBE
:104D900081F76AE070E080E090E00E94022A04C09F
:104DA00081E696E00E94962B81E696E00E946F2BAA
:104DB000892BB1F708957F928F929F92AF92BF9205
:104DC000CF92DF92EF92FF920F931F93DF93CF93D7
:104DD000CDB7DEB7AA970FB6F894DEBF0FBECDBF32
:104DE0000E94CE296B017C0181E00E94C60C04C0A8
:104DF00081E696E00E94962B81E696E00E946F2B5A
:104E0000892BB1F75F9811E032E6732E22E0822EF3
:104E1000912C8C0E9D1E5E010894A11CB11C03E018
:104E20000E94CE2920E030E06C197D098E099F098F
:104E3000693C71058105910510F021E030E0812F7A
:104E400090E028233923232BA9F10E94CE296B015E
:104E50007C01469A80ED97E00E94EC087982D401AB
:104E6000E7E2F4E089E201900D928150E1F7C5019B
:104E70006AE20E941611469880E090E00E94EC08D9
:104E8000009326040E94A50D62E370E080E090E0AC
:104E90000E94022A80912604843059F4009326044B
:104EA0008FE70E94BA0B0E94CE0B823411F410E0FF
:104EB00001C011E082E10E943E2B892B41F511E0F7
:104EC00026C05F9A469A81E696E00E94962B8D3026
:104ED000910569F08E3091051CF40A97B1F407C072
:104EE0008332910569F08234910579F40CC081E632
:104EF00096E06AE871E00E94EF2C0E94B12605C09E
:104F00000E94B91F02C00E94AD235F98469881E6B7
:104F100096E00E946F2B892B09F482CFD2CF81E6D5
:104F200096E00E946F2B04970CF181E696E00E94B8
:104F3000962B82349105D1F481E696E00E94962B5F
:104F40008E34910599F481E696E00E94962B843484
:104F5000910561F481E696E00E94962B819731F4E9
:104F600080E090E00E94EC080E94DB2608958F927A
:104F70009F92AF92BF92CF92DF92EF92FF920F93E8
:104F80001F9382E10E943E2B892B09F0ACC068EC94
:104F900070E080E090E00E94022A80E090E00E94B1
:104FA000EC080E94CE295B016C0140ECE42E42E14A
:104FB000F42E012D112DE60EF71E081F191F06C035
:104FC00082E10E943E2B892B09F085C00E94CE29E8
:104FD0006E157F058007910798F382E10E943E2BB2
:104FE000892B09F078C080ED97E00E94EC080E94C0
:104FF000CE297B018C0199249394882488E496E23D
:10500000A0E0B0E0A80EB91ECA1EDB1E29C0AE1477
:10501000BF04C006D10638F480ED97E00E94EC088A
:10502000882483941DC00E94CE296E197F09800BAD
:10503000910B693C71058105910590F00E94CE2984
:105040007B018C0180E0992009F481E0982E88236F
:1050500019F480E090E002C080ED97E00E94EC0837
:1050600082E10E943E2B892B91F280E090E00E9429
:10507000EC08882051F1809150048F5F83700E946A
:10508000691481E696E062E472E00E94682E81E68F
:1050900096E0609150044AE050E00E94F12D0E9499
:1050A0004909892B39F081E696E06FE472E00E94AD
:1050B0006B2E19C081E696E06CE672E00E94682EC5
:1050C0000E9499090E94FE130EC00E94A0240E9413
:1050D000FE130E94E11981E696E06EE872E00E94FC
:1050E0006B2E0E94DB261F910F91FF90EF90DF90B7
:1050F000CF90BF90AF909F908F900895EF92FF92C6
:105100000F931F930E94CA1286E061E00E947E2ADC
:1051100085E061E00E947E2A82E160E00E947E2AB2
:1051200084E060E00E947E2A84E061E00E940B2B14
:105130000E94D61281E696E060E072EC0E946E2B2F
:105140000E9458140E944909892B39F081E696E0A3
:105150006FE472E00E946B2E0AC081E696E06CE676
:1051600072E00E94682E0E9499090E94FE130E941C
:105170006A0E8FEF80939D050E94180978940E9413
:10518000CE297B018C0180919D058F3F09F0AFC036
:105190000E94CE296E197F09800B910B605D7740CC
:1051A0008040904008F0A3C0EECF81E696E00E94D8
:1051B000962B81E696E00E946F2B892BB1F781E652
:1051C00096E065EA72E00E94682E84E593E00E9412
:1051D000081B81E696E06CEB72E00E94682E81E687
:1051E00096E066E070E04AE050E00E94542E68ECE1
:1051F00070E080E090E00E94022A0E948F27409198
:1052000028045091290460912A0470912B04DB0139
:10521000CA010197A109B1090497A105B10568F474
:1052200040939E05433029F040E052EC61E070E08D
:1052300004C040EA56E861E070E087EF96E00E9423
:105240003A2F0E94B7275F9880E090E00E94EC0818
:105250000E946A0E80E00E94C60C809183050E9425
:10526000EF0B0E94A50D10920806109209061092ED
:105270000A066CE271E080E090E00E94022A80ED74
:1052800097E00E94EC0864E670E080E090E00E9405
:10529000022A80E090E00E94EC0810E015C064E66D
:1052A00070E080E090E00E94022A80ED97E00E948A
:1052B000EC0864E670E080E090E00E94022A80E062
:1052C00090E00E94EC081F5F80915004181738F39B
:1052D00080914F0490E084FF14C020E088719070AA
:1052E000489709F421E0822F0E9479140AC080EDCA
:1052F00097E00E94EC0882E161E00E940B2B5F9A2C
:1053000058CF1F910F91FF90EF9008951F920F9229
:105310000FB60F9211242F933F938F939F93AF93C8
:10532000BF938091180690911906A0911A06B0912A
:105330001B0630911C060196A11DB11D232F2D5F68
:105340002D3720F02D570196A11DB11D20931C066D
:105350008093180690931906A0931A06B0931B0623
:105360008091140690911506A0911606B09117062B
:105370000196A11DB11D8093140690931506A0936C
:105380001606B0931706BF91AF919F918F913F91F1
:105390002F910F900FBE0F901F9018958FB7F89414
:1053A000209118063091190640911A0650911B065B
:1053B0008FBFB901CA0108959FB7F89420911406D0
:1053C00030911506409116065091170686B5A89B98
:1053D00006C08F3F21F02F5F3F4F4F4F5F4F9FBF62
:1053E000542F432F322F2227280F311D411D511DCD
:1053F00082E0220F331F441F551F8A95D1F7B90150
:10540000CA010895EF92FF920F931F93CF93DF93FA
:105410007B018C010E94DC29EB010EC00E94DC297B
:105420006C1B7D0B685E7340C8F30894E108F108BB
:1054300001091109C851DC4FE114F10401051105FE
:1054400069F7DF91CF911F910F91FF90EF90089531
:10545000789484B5826084BD84B5816084BD85B54F
:10546000826085BD85B5816085BDEEE6F0E0808116
:1054700081608083E1E8F0E0108280818260808337
:10548000808181608083E0E8F0E0808181608083BA
:10549000E1E9F0E0808182608083808181608083A7
:1054A000E0E9F0E0808181608083E1ECF0E08081E0
:1054B000846080838081826080838081816080833A
:1054C000E3ECF0E0808181608083E0ECF0E08081BB
:1054D00082608083E2ECF0E0808181608083EAE793
:1054E000F0E080818460808380818260808380811D
:1054F000816080838081806880830895CF93DF936B
:10550000482F50E0CA018C50944FFC0134914A520C
:10551000544FFA018491882369F190E0880F991F14
:10552000FC01E455F44FA591B491FC01E654F44F0D
:10553000C591D491662351F42FB7F8948C91932F91
:10554000909589238C93888189230BC0623061F404
:105550002FB7F8948C91932F909589238C93888101
:10556000832B88832FBF06C09FB7F8948C91832B21
:105570008C939FBFDF91CF910895883071F189306E
:1055800068F4823031F1833020F4813009F042C078
:105590001DC0833089F08430E9F512C08B3059F199
:1055A0008C3028F48930E9F08A30A1F51EC08C30A7
:1055B00031F18E3079F529C0809180008F7703C05A
:1055C000809180008F7D80938000089584B58F77CF
:1055D00002C084B58F7D84BD0895809190008F773F
:1055E00007C0809190008F7D03C080919000877FDD
:1055F0008093900008958091C0008F7703C08091C0
:10560000C0008F7D8093C00008958091C200877F85
:105610008093C2000895FF920F931F93F62E482F98
:1056200050E0CA018E5E934FFC012491CA018C5058
:10563000944FFC0114914A52544FFA0104910023F3
:10564000C9F0222319F0822F0E94BD2AE02FF0E03A
:10565000EE0FFF1FE654F44FA591B4919FB7F89455
:10566000FF2021F48C911095812302C08C91812B15
:105670008C939FBF1F910F91FF9008950F931F93DD
:10568000482F50E0CA018E5E934FFC012491CA015D
:105690008C50944FFC0104914A52544FFA011491DA
:1056A000112319F420E030E015C0222319F0822FD5
:1056B0000E94BD2A812F90E0880F991F8853944F34
:1056C000FC01A591B4918C9120E030E0802311F091
:1056D00021E030E0C9011F910F91089508952091B4
:1056E0005D0630915E0680915F0690916006281BF2
:1056F000390B2F733070C901089520915D063091E8
:105700005E0680915F06909160062817390719F4AC
:105710002FEF3FEF09C0E0915F06F0916006E35E76
:10572000F94F8081282F30E0C901089520915D064E
:1057300030915E0680915F069091600628173907C8
:1057400019F42FEF3FEF13C0E0915F06F091600670
:10575000E35EF94F208180915F069091600601968B
:105760008F7390709093600680935F0630E0C9015C
:105770000895109264061092630688EE93E0A0E00C
:10578000B0E08093650690936606A0936706B09399
:10579000680687EF93E09093620680936106089510
:1057A0000F931F93DF93CF930F92CDB7DEB78C018A
:1057B00069838091B203882369F083E0BE016F5F43
:1057C0007F4F41E050E00E94CE311816190614F4C4
:1057D0009C0107C081E090E0F8019383828320E080
:1057E00030E0C9010F90CF91DF911F910F91089583
:1057F00083E00E94A5310895CF93DF9312C082E029
:105800000E9416312FEF8F3F9207C9F0E0915D069D
:10581000F0915E06E35EF94F8083D0935E06C093FD
:105820005D06C0915D06D0915E062196CF73D07063
:1058300080915F0690916006C817D90701F7DF9144
:10584000CF910895FC0180818E5F808380E86CE3B6
:105850007CE042E450E00E944C310895FC018181DB
:105860009081913A59F4813209F04CC080E06BEAA2
:1058700073E047E050E00E944C3142C0913209F0A1
:1058800041C0803239F48BEA93E067E070E00E9417
:10589000903136C0823209F035C082818093B203E4
:1058A0008091AB039091AC03A091AD03B091AE0396
:1058B000805B9440A040B04019F58091B20380FD18
:1058C00012C087E797E790930108809300082BE0C8
:1058D00088E190E00FB6F894A895809360000FBE21
:1058E000209360000DC088E10FB6F89480936000AB
:1058F000109260000FBEA895109201081092000847
:1059000081E0089580E00895CF92DF92EF92FF92B8
:105910000F931F93CF93DF937C016B018A01C0E04B
:10592000D0E00FC0D6016D916D01D701ED91FC91D2
:105930000190F081E02DC7010995C80FD91F0150D2
:1059400010400115110571F7CE01DF91CF911F9124
:105950000F91FF90EF90DF90CF900895EF92FF921C
:105960000F931F93CF93DF937C018B01C0E0D0E0B6
:10597000F8010F5F1F4F6491662359F0D701ED9135
:10598000FC910190F081E02DC7010995C80FD91F46
:10599000EFCFCE01DF91CF911F910F91FF90EF904C
:1059A0000895DC01ED91FC910190F081E02D0995C5
:1059B0000895EF92FF920F931F938C016DE00E9468
:1059C000D12C7C01C8016AE00E94D12C9C012E0DD3
:1059D0003F1DC9011F910F91FF90EF900895EF9225
:1059E000FF920F931F937C010E94AE2C8C01C70184
:1059F0000E94D92C9C01200F311FC9011F910F91CA
:105A0000FF90EF900895EF92FF920F931F937C0108
:105A10000E94D12C8C01C7010E94D92C9C01200F1F
:105A2000311FC9011F910F91FF90EF900895CF93FF
:105A3000DF93EC016115710519F420E030E00FC02F
:105A4000DB010D900020E9F71197A61BB70BE88149
:105A5000F9810280F381E02DAD0109959C01C90116
:105A6000DF91CF9108954F925F927F928F929F9294
:105A7000AF92BF92CF92DF92EF92FF920F931F935C
:105A8000DF93CF93CDB7DEB7A1970FB6F894DEBF03
:105A90000FBECDBF2C01742ECB01223008F42AE0BA
:105AA00019A231E2C32ED12CCC0EDD1E822E9924F8
:105AB000AA24BB24672D752FA50194010E9483356C
:105AC00079018A01C801B701A50194010E945135ED
:105AD000472D461B0894C108D1084A3014F4405D94
:105AE00001C0495CF6014083E114F1040105110590
:105AF00021F07E2C5F2DC801DDCFC201B6010E94CE
:105B0000172DA1960FB6F894DEBF0FBECDBFCF9173
:105B1000DF911F910F91FF90EF90DF90CF90BF909A
:105B2000AF909F908F907F905F904F900895DC0191
:105B30002115310541F4ED91FC910190F081E02DAA
:105B4000642F099508950E94332D0895EF92FF92D6
:105B50000F931F937C010E94972D8C01C7010E9417
:105B6000D92C9C01200F311FC9011F910F91FF906B
:105B7000EF900895EF92FF920F931F939A017B018C
:105B800000E010E0B801A7010E94972D1F910F912E
:105B9000FF90EF900895EF92FF920F931F937C0177
:105BA0000E94BA2D8C01C7010E94D92C9C01200FA4
:105BB000311FC9011F910F91FF90EF900895EF924F
:105BC000FF920F931F939A01E62EFF2400E010E04E
:105BD000B801A7010E94972D1F910F91FF90EF90A0
:105BE0000895EF92FF920F931F937C010E94DF2D87
:105BF0008C01C7010E94D92C9C01200F311FC901C3
:105C00001F910F91FF90EF900895CF92DF92EF9246
:105C1000FF920F931F93CF93DF93EC016A017B01F7
:105C20002115310541F4E881F9810190F081E02DE1
:105C3000642F09951BC02A303105B1F477FF13C0DA
:105C40006DE20E94D12C8C0144275527BA014C19D2
:105C50005D096E097F09CE012AE00E94332D9C0167
:105C6000200F311F04C02AE00E94332D9C01C9017E
:105C7000DF91CF911F910F91FF90EF90DF90CF9028
:105C80000895EF92FF920F931F937B019A010027D3
:105C9000F7FC0095102FB801A7010E94052E1F9157
:105CA0000F91FF90EF900895EF92FF920F931F9343
:105CB0007C010E94412E8C01C7010E94D92C9C01BD
:105CC000200F311FC9011F910F91FF90EF90089590
:105CD0000E94172D0895EF92FF920F931F937C015E
:105CE0000E94682E8C01C7010E94D92C9C01200FB4
:105CF000311FC9011F910F91FF90EF9008950895F2
:105D00001F920F920FB60F9211242F933F934F9330
:105D10008F939F93EF93FF938091C80082FD1DC0E6
:105D20004091CE002091AF063091B0062F5F3F4FDB
:105D30002F7330708091B1069091B2062817390701
:105D400071F0E091AF06F091B006E159F94F408350
:105D50003093B0062093AF0602C08091CE00FF9131
:105D6000EF919F918F914F913F912F910F900FBE87
:105D70000F901F9018951F920F920FB60F9211243B
:105D80002F933F938F939F93EF93FF932091F3066D
:105D90003091F4068091F5069091F60628173907A0
:105DA00031F48091C9008F7D8093C90014C0E091C7
:105DB000F506F091F606ED54F94F20818091F50635
:105DC0009091F60601968F7390709093F6068093EB
:105DD000F5062093CE00FF91EF919F918F913F9117
:105DE0002F910F900FBE0F901F9018958F929F923A
:105DF000AF92BF92CF92DF92EF92FF920F931F93D9
:105E0000DF93CF93CDB7DEB7FC011382128288EE09
:105E100093E0A0E0B0E084839583A683B78389E014
:105E200094E0918380837587648757874687318B99
:105E3000208B138B028BF58AE48AD78AC68AB18EAF
:105E4000A08E938E828E8F85848F8889858F898995
:105E5000868F8A89878F8B8980A3CF91DF911F914D
:105E60000F91FF90EF90DF90CF90BF90AF909F90F9
:105E70008F900895AF92BF92DF92EF92FF920F93AF
:105E80001F93CF93DF93EC017A018B01DD24403027
:105E900081EE580780E0680780E0780711F0DD2484
:105EA000D39491E0A92EB12CEC89FD89DD2069F015
:105EB000C50108A002C0880F991F0A94E2F78083E9
:105EC00060E079E08DE390E005C0108260E874E85E
:105ED0008EE190E0A80197010E9483352150304067
:105EE00040405040569547953795279580E12030A2
:105EF000380720F0DD2011F0DD24D6CFE889F989BC
:105F00003083EA89FB89208319A2EE89FF894081C9
:105F100021E030E0C9010C8C02C0880F991F0A945F
:105F2000E2F7482B4083EE89FF894081C9010D8C3F
:105F300002C0880F991F0A94E2F7482B4083EE892C
:105F4000FF894081C9010E8C02C0880F991F0A94F5
:105F5000E2F7482B4083EE89FF8980810F8C02C0D5
:105F6000220F331F0A94E2F7209528232083DF9124
:105F7000CF911F910F91FF90EF90DF90BF90AF9066
:105F80000895DC011C96ED91FC911D97E05CFF4F9C
:105F90002191319180819181281B390B2F733070B1
:105FA000C901089587EF96E00E94C12F892B11F057
:105FB0000E947F2E0895DC011C96ED91FC911D97A7
:105FC000E05CFF4F20813181E054F040DF01AE5BA7
:105FD000BF4F8D919C9111972817390719F42FEF16
:105FE0003FEF07C08D919C91E80FF91F8081282F0A
:105FF00030E0C9010895DC011C96ED91FC911D97DC
:10600000E05CFF4F20813181E054F040DF01AE5B66
:10601000BF4F8D919C9111972817390719F42FEFD5
:106020003FEF10C08D919C911197E80FF91F2081CF
:106030008D919C91119701968F73907011969C93FE
:106040008E9330E0C9010895DC0191968C9191976F
:10605000882339F05496ED91FC915597808186FF05
:10606000F9CF91961C920895CF93DF93EC01EE85C2
:10607000FF85E05CFF4F20813181E054F0402F5FCD
:106080003F4F2F733070DF01AE5BBF4F8D919C91FE
:10609000119728173907D1F3E05CFF4F8081918178
:1060A000E054F040E80FF91F6083EE85FF85E05C67
:1060B000FF4F31832083EE89FF89208181E090E0CA
:1060C0000F8C02C0880F991F0A94E2F7282B2083B7
:1060D00081E089A3EC89FD8980818064808381E0EF
:1060E00090E0DF91CF9108958F929F92AF92BF92EF
:1060F000CF92DF92EF92FF920F931F9300D000D0C8
:106100000F92EDB7FEB7319684E0ADB7BEB71196EA
:106110008C9383E0818387E0828385E0838381E0C1
:10612000848387EF96E06FE676E043EB56E02DEC54
:1061300030E00CEC10E0B8ECEB2EF12CA9ECCA2E00
:10614000D12CFAECAF2EB12CEEEC8E2E912C0E94BD
:10615000F62E0F900F900F900F900F901F910F91B0
:10616000FF90EF90DF90CF90BF90AF909F908F9077
:106170000895CF93DF930E94282A81E297E00E943E
:10618000B0310E947E28C2EDDFE20E94E514209724
:10619000E1F30E94D22FF9CFFC0104C08091F100FD
:1061A000819361506623D1F7289884E680931A077B
:1061B00008959FB7F89487708093E9008091F2006A
:1061C0009FBF0895282F80911B078823C1F057FF98
:1061D0001AC015C0289890931A078091F1008193F6
:1061E000E217F307B9F74115510539F08091F20034
:1061F000882319F48BE68093E800AFBF02C04FEF0D
:106200005FEFCA010895AFB7F89427702093E900B3
:106210008091F200282F30E0241735070CF4A901F3
:10622000FB019B01240F311D94E6DACFDF93CF935E
:106230000F92CDB7DEB7BE016F5F7F4F41E050E0F8
:106240000E94E230019719F02FEF3FEF03C08981E0
:10625000282F30E0C9010F90CF91DF9108952FB71B
:10626000F89487708093E9008091E80085FD02C072
:1062700090E004C08091F20090E4981B2FBF892F1A
:1062800008951092E90010921D0710921C07909338
:106290001F0780931E070895FF920F931F93F82EF8
:1062A000142F052F40911E0750911F07212F302FCB
:1062B000C901DC01FB016EEF29C0F7FE02C0949119
:1062C00001C0908120911C0730911D0724173507CC
:1062D000ACF48091E8008570E1F38091E80082FFE2
:1062E00003C02FEF3FEF17C09093F100C901019653
:1062F0008F739070892B11F46093E8002F5F3F4FEC
:1063000030931D0720931C07119731961097A9F61B
:10631000812F902F9C01C9011F910F91FF9008952B
:106320000F931F939C01162F072F8091E80082FF87
:10633000FCCFC901612F0E94CC308BEF8093E80025
:10634000812F902F1F910F9108958093E9008091E4
:10635000F200882319F08AE38093E80008950895F5
:1063600010921B0781E08093D70080EA8093D800C9
:1063700082E189BD09B400FEFDCF61E070E080E0FC
:1063800090E00E94022A80E98093D8008CE08093FC
:10639000E2001092E000559A209A08956F927F9241
:1063A0008F929F92AF92BF92CF92DF92EF92FF9225
:1063B0000F931F93CF93DF93E82E942E852E809119
:1063C0001B07882309F18B01242F352FC901EC010C
:1063D0006AEFF62E57E0752E7E208E2D90E040E27B
:1063E000A42EB12CA822B9223AE3632E20E4C22EB7
:1063F000D12CC822D9224CC08E2D0E942F31282F9B
:10640000882361F4FA9419F42FEF3FEF4CC061E058
:1064100070E080E090E00E94022A3AC090E0C81745
:10642000D9070CF42C2FC21BD1094FB7F8947092E6
:10643000E900A114B10421F406C01092F10021502A
:106440002223D9F719C0E7FC03C0F801922F10C02E
:10645000C801322F06C0FC010196E491E093F100DF
:1064600031503323C1F706C081918093F1009150E0
:106470009923D1F7020F111D8091E80085FF05C017
:10648000209729F4C114D10411F06092E8004FBFA5
:10649000209709F0B1CF5D9884E680931907292DE4
:1064A000382DC9019C01C901DF91CF911F910F9136
:1064B000FF90EF90DF90CF90BF90AF909F908F9024
:1064C0007F906F9008951F920F920FB60F92112434
:1064D0002F933F934F935F936F937F938F939F93EC
:1064E000AF93BF93EF93FF938091E1001092E1008F
:1064F000982F93FF0FC01092E90081E08093EB008A
:106500001092EC0082E38093ED0010921B0788E06C
:106510008093F00092FF28C083E00E94A53182E0C2
:106520000E94D930882321F081E696E00E94FC2B5E
:1065300080911907882351F0809119078150809329
:10654000190780911907882309F45D9A80911A0729
:10655000882351F080911A07815080931A07809107
:106560001A07882309F4289AFF91EF91BF91AF9100
:106570009F918F917F916F915F914F913F912F915B
:106580000F900FBE0F901F9018950F931F93DF93DE
:10659000CF930F92CDB7DEB719828E010F5F1F4FD9
:1065A000C8010E94222CC8010E944535898190E0D3
:1065B0000F90CF91DF911F910F9108951F920F922D
:1065C0000FB60F921124CF92DF92EF92FF920F93AA
:1065D0002F933F934F935F936F937F938F939F93EB
:1065E000AF93BF93EF93FF93DF93CF93CDB7DEB716
:1065F0006197DEBFCDBF1092E9008091E80083FF74
:10660000EBC0CE01019668E00E94CC3082EF80930F
:10661000E800998197FF05C08091E80080FFFCCFDA
:1066200003C08EEF8093E800292F30E0C901807607
:106630009070892B09F0B1C08A81882329F41092C7
:10664000F1001092F100BDC0813009F4BAC083306E
:1066500009F4B7C0853049F48091E80080FFFCCF91
:106660008B8180688093E300ACC0863009F06BC0FA
:106670000C81EF80F884023071F580E090E00E9498
:1066800041310E94C53299E079E0C72ED12CCC0E61
:10669000DD1EF601292F11922A95E9F799870A87BD
:1066A00091E09E8790E8988B9AEF998B20911C0738
:1066B00030911D07275F3F4F3C872B878D87C70190
:1066C0000E94413180E0B60149E050E00E944C3127
:1066D0000E94C53276C0C7010E944131023241F4A6
:1066E00082E290E00E943D35892B09F46EC069C0BA
:1066F000013079F48F819885089719F481E08093AF
:10670000200780912007882309F063C0ECEBFCE0B0
:1067100013C0033009F059C08B81882319F4EEE7C8
:10672000FCE00AC0823019F4E2E8FCE005C08130E8
:1067300009F04BC0E4EAFCE0449180E8BF0150E07E
:106740000E944C313EC0873009F43FC0883021F4AC
:1067500081E08093F10035C0893099F52370307065
:10676000232B99F5E1EEFCE091E031E026E39093F4
:10677000E9003093EB0084918093EC002093ED00CE
:106780009F5F3196953099F78EE78093EA001092DB
:10679000EA008B8180931B0714C08F8198850E942B
:1067A00041318D81882329F4CE0101960E942E2C3F
:1067B00006C0823051F4CE0101960E94073488232E
:1067C00021F08EEF8093E80007C081E28093EB0018
:1067D00003C0EEECFCE0B0CF6196DEBFCDBFCF9141
:1067E000DF91FF91EF91BF91AF919F918F917F9139
:1067F0006F915F914F913F912F910F91FF90EF908B
:10680000DF90CF900F900FBE0F901F901895FC0156
:1068100091818081813A31F4913089F080E0933028
:1068200089F40DC0813269F49B3021F48281809318
:10683000B30305C09A3029F482818093B40381E0C8
:10684000089580E00895FC0110820895FC011382F0
:10685000128289E194E0918380830895EF92FF9200
:106860000F931F938C01E62EDC01ED91FC910480C7
:10687000F581E02D0995F82ED801ED91FC91068067
:10688000F781E02DC8016E2D09958F2D90E01F91A5
:106890000F91FF90EF90089582E297E00E942334D9
:1068A00083E297E00E9426340895EF92FF920F93BF
:1068B0001F93DF93CF930F92CDB7DEB789838B0100
:1068C0007A0184E0BE016F5F7F4F41E050E00E949B
:1068D000CE3184E4B801A7010E94CE310F90CF9150
:1068E000DF911F910F91FF90EF90089582E048E0B3
:1068F00050E00E9455340895FC01168217821086DC
:1069000011861286138614823496BF010E94763453
:106910000895DC01683810F0685829C0E62FF0E0CF
:1069200067FF13C0E058F04081E090E002C0880F9C
:10693000991FEA95E2F7809514962C9114972823D5
:1069400014962C93149760E012C0ED59F24F6491A5
:10695000662319F420E030E01DC067FF08C01496DC
:106960008C9114978D7F14968C9314976F77FD01FB
:1069700090E0662321F08681861709F416829F5FD6
:1069800031969630B1F7CD011496BD010E94763450
:1069900021E030E0C9010895CF93DF93DC0168382E
:1069A00010F0685825C0E62FF0E067FF12C0E058ED
:1069B000F04081E090E002C0880F991FEA95E2F76D
:1069C00014962C911497282B14962C93149760E00E
:1069D0000FC0ED59F24F64916623D9F167FF08C0EB
:1069E00014968C911497826014968C9314976F77F9
:1069F00016968C9116978617A9F117968C91179772
:106A0000861781F118968C911897861759F1199667
:106A10008C911997861731F11A968C911A978617CF
:106A200009F11B968C911B978617E1F0ED01E0E0D0
:106A3000F0E09E2F8E81882321F4EA0FFB1F6683EE
:106A400006C09F5F31962196E630F10591F79630AA
:106A500049F481E090E013969C938E93129720E086
:106A600030E007C0CD011496BD010E94763421E0CC
:106A700030E0C901DF91CF91089580E865EE7CE0B8
:106A800045E650E00E944C310895FC0180818F5F03
:106A9000808380E86AE47DE049E150E00E944C3167
:106AA0000895629FD001739FF001829FE00DF11D58
:106AB000649FE00DF11D929FF00D839FF00D749F78
:106AC000F00D659FF00D9927729FB00DE11DF91F24
:106AD000639FB00DE11DF91FBD01CF011124089581
:106AE00097FB092E07260AD077FD04D049D006D09F
:106AF00000201AF4709561957F4F0895F6F79095F0
:106B000081959F4F0895A1E21A2EAA1BBB1BFD0180
:106B10000DC0AA1FBB1FEE1FFF1FA217B307E4077C
:106B2000F50720F0A21BB30BE40BF50B661F771FD4
:106B3000881F991F1A9469F76095709580959095B4
:106B40009B01AC01BD01CF01089597FB092E0526DD
:106B50000ED057FD04D0D7DF0AD0001C38F4509572
:106B60004095309521953F4F4F4F5F4F0895F6F771
:106B700090958095709561957F4F8F4F9F4F0895A9
:106B8000AA1BBB1B51E107C0AA1FBB1FA617B70753
:106B900010F0A61BB70B881F991F5A95A9F780956F
:106BA0009095BC01CD010895EE0FFF1F0590F49163
:106BB000E02D0994911106C0803219F0895085505A
:106BC000D0F708959927882708952F923F924F92E2
:106BD0005F926F927F928F929F92AF92BF92CF926D
:106BE000DF92EF92FF920F931F93CF93DF93CDB776
:106BF000DEB7CA1BDB0B0FB6F894DEBF0FBECDBFEE
:106C000009942A88398848885F846E847D848C84BE
:106C10009B84AA84B984C884DF80EE80FD800C81C7
:106C20001B81AA81B981CE0FD11D0FB6F894DEBFAA
:0C6C30000FBECDBFED010895F894FFCF1A
:106C3C004E6F005965730054582074696D656F75FB
:106C4C007421006D6F64756C65206C6F636B65648B
:106C5C003F00486F70206368616E6E656C20002089
:106C6C0040200053004E2F4100386368002C002C4C
:106C7C00205B005D20280029004E4F5420454E41DA
:106C8C00424C45440053656E64696E6720736574AD
:106C9C0074696E677320746F2052580A00526573C2
:106CAC00657474696E672073657474696E6773209C
:106CBC006F6E2052580A0041626F727465642065D1
:106CCC00646974730A00696E76616C69642073651B
:106CDC006C656374696F6E000D0A496E76616C6940
:106CEC006420696E707574202D2064697363617201
:106CFC006465642107007363616E6E6572206D6F4D
:106D0C0064650053657474696E677320736176658E
:106D1C006420746F20454550524F4D0A00526576E1
:106D2C0065727465642073657474696E677320662C
:106D3C00726F6D20454550524F4D0A004C6F616487
:106D4C00656420666163746F727920646566617531
:106D5C006C74730A004B657920616E642063686102
:106D6C006E6E656C732072616E646F6D697A6564AA
:106D7C000A004E65772070726F66696C653A004C3C
:106D8C006F616465642073657474696E67732066E3
:106D9C00726F6D20454550524F4D0A00454550527B
:106DAC004F4D2064617461206E6F742076616C6944
:106DBC00642C207265696E6974696E670A00456E91
:106DCC00746572696E672062696E64696E67206DA6
:106DDC006F64650A004F70656E4C52536E67205499
:106DEC0058207374617274696E672000206F6E2076
:106DFC004857200050504D005253534900534441C2
:106E0C000053434C00525844005458440041494EDE
:106E1C00004C424545500053504B54524D00534288
:106E2C0055530053554D44004C4C494E44000034CE
:106E3C002B34003800382B340031320031322B34F3
:106E4C000031360001000000C01200001A400AA1F7
:106E5C00204EA5001B1E27522C2330802500000538
:106E6C00400AA1204EA50020244EA52C2330004B17
:106E7C00000006400AD0009D49007B289D492C2328
:106E8C003000E1000005400A4501D7DC03B81E0EB6
:106E9C00BF00232E48E801008A400A6001555502C4
:106EAC00AD1E20000023C88025000005400AA1204B
:106EBC004EA50020244EA52C233000020002000217
:106ECC0000020002000200020002000200020002A6
:106EDC0000020002000200020002FF00E1000000BC
:106EEC000000000101C402C802CD02D102D502D9B2
:106EFC0002DD02E102E702EE02F302F802FE02FEFC
:106F0C0002FE02FE023501FF020303050309030C16
:106F1C00031103350100070B0C10111500160A1391
:106F2C0022312900000000D02B842C6F2B962B7D56
:106F3C002BF82BFC2B000000003430842CC12FFBD1
:106F4C002FDB2F2430000000002E34842CCC34890D
:046F5C00347C34004D
:00000001FF
